:100000000084FF1F11040000A10D0000A10D0000DD
:10001000A10D0000A10D0000A10D0000A10D000028
:10002000A10D0000A10D0000A10D0000E11D0000C8
:10003000A10D0000A10D0000A10D0000912C0000F9
:10004000A10D0000A10D0000A10D0000A10D0000F8
:10005000A10D0000A10D0000A10D0000A10D0000E8
:10006000A10D0000A10D0000A10D0000A10D0000D8
:10007000A10D0000A10D0000A10D0000A10D0000C8
:10008000A10D0000A10D0000A10D0000A10D0000B8
:10009000A10D0000A10D0000A10D0000A10D0000A8
:1000A000A10D0000A10D0000A10D0000A10D000098
:1000B000A10D0000A10D0000A10D0000A10D000088
:1000C000A10D0000A10D0000A10D0000A10D000078
:1000D000A10D0000A10D0000A10D0000A10D000068
:1000E000A10D0000A10D0000A10D0000A10D000058
:1000F000A10D0000A10D0000A10D0000A10D000048
:10010000A10D0000A10D0000A10D0000A10D000037
:10011000A10D0000A10D0000A10D0000A10D000027
:10012000A10D0000A10D0000A10D0000A10D000017
:10013000A10D0000A10D0000A10D0000A10D000007
:10014000A10D0000A10D0000A10D0000A10D0000F7
:10015000A10D0000A10D0000A10D0000A10D0000E7
:10016000A10D0000C12D0000A10D0000A10D000097
:10017000A10D0000A10D0000A10D0000A10D0000C7
:10018000A10D0000A10D0000A10D0000A10D0000B7
:10019000A10D000051760000A10D0000A10D00008E
:1001A000A10D0000A10D0000A10D0000A10D000097
:1001B000A10D0000A10D0000A10D0000A10D000087
:10040000FFFFFFFFFFFFFFFFFFFFFFFF7EFFFFFF7D
:1004100072B6254880F3098824484EF60851CEF27A
:1004200000010860022080F31488BFF36F8F00F092
:1004300077FC03F05DF81E481E491F4A91423CBFFD
:1004400041F8040BFAE71D49174A91423CBF41F8B5
:10045000040BFAE71A491B4A1B4B9A423EBF51F85C
:10046000040B42F8040BF8E700201849184A91429F
:100470003CBF41F8040BFAE700F06AFC00F058FCBE
:10048000144C154DAC4203DA54F8041B8847F9E7C5
:1004900003F00EFD114C124DAC4203DA54F8041B6C
:1004A0008847F9E700F04CBC0086FF1F0000000001
:1004B000555555550080FF1F0084FF1F0084FF1F06
:1004C000A08A00000086FF1F4086FF1F0088FF1FD4
:1004D0002494FF1F1004000010040000100400000A
:1004E00010040000000000000000000000000000F8
:1004F0002DE9F04FC1F80CD0C3689D46BDE8F08FE0
:1005000000F00EFD002383F311882846A047002049
:1005100001F026F900F0F4FC00F092FF00F000FD7D
:1005200000DFFEE700000000000000000000000007
:1005300081F0004102E000BF83F0004330B54FEA94
:1005400041044FEA430594EA050F08BF90EA020F01
:100550001FBF54EA000C55EA020C7FEA645C7FEA94
:10056000655C00F0E2804FEA5454D4EB5555B8BFB7
:100570006D420CDD2C4480EA020281EA030382EA28
:10058000000083EA010180EA020281EA0303362DBA
:1005900088BF30BD11F0004F4FEA01314FF4801C8D
:1005A0004CEA113102D0404261EB410113F0004F9F
:1005B0004FEA03334CEA133302D0524263EB430356
:1005C00094EA050F00F0A780A4F10104D5F1200EF4
:1005D0000DDB02FA0EFC22FA05F2801841F100014F
:1005E00003FA0EF2801843FA05F359410EE0A5F123
:1005F00020050EF1200E012A03FA0EFC28BF4CF054
:10060000020C43FA05F3C01851EBE37101F0004509
:1006100007D54FF0000EDCF1000C7EEB00006EEB16
:100620000101B1F5801F1BD3B1F5001F0CD34908A0
:100630005FEA30004FEA3C0C04F101044FEA4452F7
:1006400012F5800F80F09A80BCF1004F08BF5FEA7E
:10065000500C50F1000041EB045141EA050130BD5E
:100660005FEA4C0C404141EB010111F4801FA4F101
:100670000104E9D191F0000F04BF01460020B1FA56
:1006800081F308BF2033A3F10B03B3F120020CDA8E
:100690000C3208DD02F1140CC2F10C0201FA0CF06C
:1006A00021FA02F10CE002F11402D8BFC2F1200CD1
:1006B00001FA02F120FA0CFCDCBF41EA0C01904087
:1006C000E41AA2BF01EB0451294330BD6FEA0404D0
:1006D0001F3C1CDA0C340EDC04F11404C4F12002BB
:1006E00020FA04F001FA02F340EA030021FA04F3CD
:1006F00045EA030130BDC4F10C04C4F1200220FA24
:1007000002F001FA04F340EA0300294630BD21FA61
:1007100004F0294630BD94F0000F83F4801306BF27
:1007200081F480110134013D4EE77FEA645C18BF1B
:100730007FEA655C29D094EA050F08BF90EA020FB2
:1007400005D054EA000C04BF1946104630BD91EAAA
:10075000030F1EBF0021002030BD5FEA545C05D1AD
:100760004000494128BF41F0004130BD14F58004EC
:100770003CBF01F5801130BD01F0004545F0FE4160
:1007800041F470014FF0000030BD7FEA645C1ABF95
:10079000194610467FEA655C1CBF0B46024650EACC
:1007A000013406BF52EA033591EA030F41F40021F8
:1007B00030BD00BF90F0000F04BF0021704730B57E
:1007C0004FF4806404F132044FF000054FF0000153
:1007D00050E700BF90F0000F04BF0021704730B514
:1007E0004FF4806404F1320410F0004548BF4042E9
:1007F0004FF000013EE700BF42004FEAE2014FEA3E
:1008000031014FEA02701FBF12F07F4393F07F4F18
:1008100081F06051704792F0000F14BF93F07F4F4A
:10082000704730B54FF4607401F0004521F000418D
:1008300020E700BF50EA010208BF704730B54FF013
:1008400000050AE050EA010208BF704730B511F018
:10085000004502D5404261EB41014FF4806404F150
:1008600032045FEA915C3FF4DCAE4FF003025FEAD2
:10087000DC0C18BF03325FEADC0C18BF033202EB5A
:10088000DC02C2F1200300FA03FC20FA02F001FAB4
:1008900003FE40EA0E0021FA02F11444C1E600BF53
:1008A00070B54FF0FF0C4CF4E06C1CEA11541DBF06
:1008B0001CEA135594EA0C0F95EA0C0F00F0DEF8D1
:1008C0002C4481EA030621EA4C5123EA4C5350EAB6
:1008D000013518BF52EA033541F4801143F4801307
:1008E00038D0A0FB02CE4FF00005E1FB02E506F098
:1008F0000042E0FB03E54FF00006E1FB03569CF0ED
:10090000000F18BF4EF0010EA4F1FF04B6F5007FF2
:1009100064F5407404D25FEA4E0E6D4146EB060664
:1009200042EAC62141EA55514FEAC52040EA5E50ED
:100930004FEACE2EB4F1FD0C88BFBCF5E06F1ED897
:10094000BEF1004F08BF5FEA500E50F1000041EBCE
:10095000045170BD06F0004646EA010140EA02007B
:1009600081EA0301B4EB5C04C2BFD4EB0C0541EA9D
:10097000045170BD41F480114FF0000E013C00F3B2
:10098000AB8014F1360FDEBF002001F0004170BDD6
:10099000C4F10004203C35DA0C341BDC04F11404EF
:1009A000C4F1200500FA05F320FA04F001FA05F27B
:1009B00040EA020001F0004221F0004110EBD37048
:1009C00021FA04F642EB06015EEA430E08BF20EA74
:1009D000D37070BDC4F10C04C4F1200500FA04F317
:1009E00020FA05F001FA04F240EA020001F00041A9
:1009F00010EBD37041F100015EEA430E08BF20EA1C
:100A0000D37070BDC4F1200500FA05F24EEA020E63
:100A100020FA04F301FA05F243EA020321FA04F092
:100A200001F0004121FA04F220EA020000EBD37049
:100A30005EEA430E08BF20EAD37070BD94F0000F49
:100A40000FD101F00046400041EB010111F4801F7D
:100A500008BF013CF7D041EA060195F0000F18BF2E
:100A6000704703F00046520043EB030313F4801F6A
:100A700008BF013DF7D043EA0603704794EA0C0F24
:100A80000CEA135518BF95EA0C0F0CD050EA41063A
:100A900018BF52EA4306D1D181EA030101F00041B7
:100AA0004FF0000070BD50EA410606BF10461946DF
:100AB00052EA430619D094EA0C0F02D150EA0136EB
:100AC00013D195EA0C0F05D152EA03361CBF10462C
:100AD00019460AD181EA030101F0004141F0FE41CB
:100AE00041F470014FF0000070BD41F0FE4141F44F
:100AF000780170BD70B54FF0FF0C4CF4E06C1CEA4F
:100B000011541DBF1CEA135594EA0C0F95EA0C0F03
:100B100000F0A7F8A4EB050481EA030E52EA0335BE
:100B20004FEA013100F088804FEA03334FF08055DF
:100B300045EA131343EA12634FEA022245EA11150C
:100B400045EA10654FEA00260EF000419D4208BFBD
:100B5000964244F1FD0404F5407402D25B084FEA6A
:100B60003202B61A65EB03055B084FEA32024FF416
:100B700080104FF4002CB6EB020E75EB030E22BF73
:100B8000B61A754640EA0C005B084FEA3202B6EB33
:100B9000020E75EB030E22BFB61A754640EA5C00E2
:100BA0005B084FEA3202B6EB020E75EB030E22BF72
:100BB000B61A754640EA9C005B084FEA3202B6EB73
:100BC000020E75EB030E22BFB61A754640EADC0032
:100BD00055EA060E18D04FEA051545EA16754FEA94
:100BE00006164FEAC30343EA52734FEAC2025FEAB2
:100BF0001C1CC0D111F4801F0BD141EA00014FF041
:100C000000004FF0004CB6E711F4801F04BF014311
:100C10000020B4F1FD0C88BFBCF5E06F3FF6AFAE2D
:100C2000B5EB030C04BFB6EB020C5FEA500C50F1BD
:100C3000000041EB045170BD0EF0004E4EEA113140
:100C400014EB5C04C2BFD4EB0C0541EA045170BD47
:100C500041F480114FF0000E013C90E645EA060E8B
:100C60008DE60CEA135594EA0C0F08BF95EA0C0FB9
:100C70003FF43BAF94EA0C0F0AD150EA01347FF401
:100C800034AF95EA0C0F7FF425AF104619462CE7D8
:100C900095EA0C0F06D152EA03353FF4FDAE10463B
:100CA000194622E750EA410618BF52EA43067FF48C
:100CB000C5AE50EA41047FF40DAF52EA43057FF41C
:100CC000EBAE12E700000000000000000000000092
:100CD0004FEA410212F5001215D211D56FF4787364
:100CE000B3EB625212D94FEAC12343F0004343EA07
:100CF000505311F0004F23FA02F018BF40427047E2
:100D00004FF00000704750EA013005D111F000406B
:100D100008BF6FF0004070474FF00000704700BF01
:100D2000704700BF0000000000000000000000004D
:100D3000704700BF0000000000000000000000003D
:100D4000FEE700BF000000000000000000000000FF
:100D5000F0B4114E002506F1800796E81A00A34270
:100D60000DD204391A4651F8040F42F8040BA2427E
:100D7000F9D3DA43144424F0030404342344F2681E
:100D8000934203D243F8045B9342FBD31036BE4236
:100D9000E3D3F0BC704700BFFC7700000000000008
:100DA000FEE700BF0000000000000000000000009F
:100DB00030BFFDE700000000000000000000000060
:100DC000F8B51C4C1C4E002500F0AAF900F040F9C3
:100DD0002563656300F0E4FE00F042FF04F1380093
:100DE0001649802200F05CFB154B1649012280F861
:100DF0002020DF68144AC1614FF6FF0139400A43E1
:100E0000DA60F2681149A06142F08072F2600A680B
:100E1000202042F0010210240A60DC7783F82200CF
:100E200000F05EF885F3118862B60948BDE8F84025
:100E300000F0CEBBD888FF1FF0ED00E0DC790000A9
:100E400000ED00E00084FF1F0003FA05001000E041
:100E50007C7800000000000000000000000000009E
:100E600072B6014BD862FEE7D888FF1F0000000071
:100E70002DE9F843174E00F0CBF8B26992F8233011
:100E800013B1013B82F8233000F0C2F8124FB36A6D
:100E9000F4690133BC42B36219D0A568013DA56075
:100EA000ADB94FF020092368D4F80C80E5605F608D
:100EB000F36100F065F885F311882069C04789F374
:100EC000118800F045F8F469A368002BEBD0BDE869
:100ED000F88300BFD888FF1FF488FF1F00000000C0
:100EE000044B1A6B0AB95B6B13B10348FFF7B8BF29
:100EF000704700BFD888FF1FAC78000000000000DA
:100F000010B5054C236B0BB9636B13B10348FFF7A6
:100F1000A7FF0123636310BDD888FF1FB4780000CA
:100F200010B5074C236B2BB9636B002B02DD00233C
:100F3000636310BD0348FFF793FF0023636310BD95
:100F4000D888FF1FBC7800000000000000000000EF
:100F500010B5064C236B002B01DD636B13B1044805
:100F6000FFF77EFF0123636310BD00BFD888FF1F1A
:100F7000C478000000000000000000000000000035
:100F800010B5084C236B002B05DD636B002B02DDD5
:100F90000023636310BD0448FFF762FF002363630F
:100FA00010BD00BFD888FF1FCC78000000000000F3
:100FB00010B5202383F31188074C236B002B01DB32
:100FC000626B1AB10548FFF74BFF236B01332363B4
:100FD000002383F3118810BDD888FF1FD478000048
:100FE00010B5202383F31188074C236B002B01DD00
:100FF000626B1AB10548FFF733FF236B013B236394
:10100000002383F3118810BDD888FF1FDC7800000F
:10101000054B1A6B002A03DB5B6B002B00DD70476E
:101020000248FFF71DBF00BFD888FF1FE47800000B
:10103000044B1A6B1AB95B6B002B00DD704702483A
:10104000FFF70EBFD888FF1FEC78000000000000FB
:10105000054B4FF0FF3003F11C02002158629962EA
:10106000DA611A62704700BFD888FF1F00000000D5
:10107000F8B505460C4616461F46FFF7C9FFD5B121
:10108000CEB1C4B10E482F61C369EE609A68944234
:1010900004D91B68A41A9A68A242FAD35A686A60F3
:1010A0002B6015605D60AC6099684FF0FF32091BE2
:1010B00099604262F8BD0348FFF7D2FEE2E700BF45
:1010C000D888FF1FF4780000000000000000000036
:1010D00038B50446FFF79CFFACB1E3687BB12368E9
:1010E000A2689D6861680A482A449A600B60256876
:1010F00000224FF0FF336960E260436238BD05486B
:10110000FFF7AEFEEBE70348FFF7AAFEE5E700BFF7
:10111000D888FF1F007900000000000000000000D8
:10112000034B00221B605B601B615B619A60704730
:10113000D888FF1F00000000000000000000000031
:1011400010B50446FFF764FFC4B194F820308BB1AA
:101150000F2B0FD00022A1680A4B84F820201B68B7
:101160009A688A42FBD25A68626023602046146003
:101170005C6010BD0448FFF773FEEBE70248FFF721
:101180006FFEE2E7D888FF1F107900000000000022
:1011900038B50446202383F31188FFF7D9FE94F86D
:1011A0002030072B10D8DFE803F0150F0F1B0A04BF
:1011B0000F0A656AFFF72CFFAB680133AB6094E858
:1011C0000C001A60226853604FF0FF3363622046C0
:1011D000FFF7B6FFFFF7D4FE002383F3118838BD75
:1011E000636A00221A604FF0FF3363622046FFF704
:1011F000A7FFEFE700000000000000000000000073
:1012000010B50446FFF704FFC4B194F820308BB149
:101210000F2B0FD00022A1680A4B84F820201B68F6
:101220009A688A42FBD85A6862602360204614603C
:101230005C6010BD0448FFF713FEEBE70248FFF7C0
:101240000FFEE2E7D888FF1F1C79000000000000B5
:1012500070B5134C0646A569FFF7EAFE236885F8CA
:1012600020601A6822601420012185F82300546050
:10127000A36183F82010EFF30982E969243A9142CF
:1012800005D829461846BDE87040FFF731B9054832
:10129000FFF7E6FDA0692946BDE87040FFF728B9D1
:1012A000D888FF1F30790000000000000000000017
:1012B00070B50C4686B00646FFF7BAFE631C14D024
:1012C0000E4D0F4AAB69214601A8FFF7D1FE30460B
:1012D000FFF7BEFFFFF79CFE049B13B101A8FFF7C9
:1012E000F7FEAB69586A06B070BD044D3046FFF793
:1012F000AFFFAB69586A06B070BD00BFD888FF1F4A
:10130000911100000000000000000000000000003B
:10131000F8B51C4C05460F46A669FFF789FE236801
:10132000A34204D0A2699B6892689A421DD3B36815
:10133000AA686F629A4213D93046FFF701FF012372
:101340000646A56185F82030EFF30983C269243B86
:101350009A420ED828463146BDE8F840FFF7C8B893
:101360002846BDE8F840FFF7EBBE0748FFF778FDD9
:10137000DDE70648FFF774FD28463146BDE8F84032
:10138000FFF7B6B8D888FF1F407900003079000019
:10139000084B9A691B6892F823109B68906821B9E2
:1013A000834234BF002001207047834294BF002055
:1013B00001207047D888FF1F0000000000000000D7
:1013C00038B50E4C2368A0691A6822600121546068
:1013D00083F82010A361FFF713FF0546EFF309839D
:1013E000C269243B9A4202D90548FFF739FDA0693A
:1013F0002946BDE83840FFF77BB800BFD888FF1FFB
:101400003079000000000000000000000000000033
:1014100008B5FFF70DFEFFF7FBFD064B1A689B6949
:1014200092689B689A4200D808BDBDE80840FFF763
:10143000C7BF00BFD888FF1F0000000000000000E9
:1014400038B5134C2368A0691A6893F823102260FA
:1014500001255460A36183F82050A1B9FFF770FE05
:101460001423054680F82330EFF30983EA69243B0F
:101470009A4202D90748FFF7F3FCA0692946BDE864
:101480003840FFF735B8FFF7BBFE0546ECE700BF75
:10149000D888FF1F30790000000000000000000025
:1014A0002DE9F043114CC26367694761002500F1E3
:1014B0002C064FF002094FF014084FF0010C00F118
:1014C000280E82600461816180F8209080F823807A
:1014D00080F822C080F821508563456338616061DF
:1014E000C0F828E0C6620663BDE8F083D888FF1F15
:1014F0002DE9F8430446FFF78BFD002C5BD06368B1
:10150000580702D1A268510749D02D48FFF7A8FC1F
:10151000E268FF2A49D82569002D46D0A368606893
:1015200066692468274943F8304C43F82C0C4FF087
:10153000020C00204FF0140E012403F8264C03F88F
:10154000270C03F828CC03F825EC4F6943F8686CA6
:1015500043F86C5CA3F14804A3F11C05DFF8688034
:1015600043F8100CA3F16C09A3F1200643F8140C06
:1015700043F8402C43F80C2C43F83C9C43F84C8C2B
:1015800043F8381C43F8347C20463C614C6143F8F6
:10159000206C43F81C5C43F8185CBDE8F883934268
:1015A000B3D2D31AC72BB3D8AFE70548FFF758FC1F
:1015B0002569E268B2E70248FFF752FC9FE700BFE7
:1015C0007C790000D888FF1F0105000000000000A2
:1015D00010B50446406800F0BBF910B11548FFF79C
:1015E0003FFC6368A268934238BF552103D203F8D9
:1015F000011B9342FBD1202383F31188FFF780FC6A
:101600002046FFF775FF00210446FFF781FEFFF734
:1016100087FC094B1A689A4207D0996993688A68CF
:101620009A4202D20548FFF71BFC002383F311887E
:10163000204610BDB4790000D888FF1FD079000083
:1016400010B52023044683F31188FFF759FC94F862
:101650002230EBB1013B84F82230236A03F0FF1300
:101660000F2B1BD0FFF75CFC224B1A689A4204D068
:10167000996993688A689A4203D3002383F3118897
:1016800010BD1D48FFF7ECFB002383F3118810BD4C
:101690001A48FFF7E5FB94F82230DBE7636922691B
:1016A0001A6122695361FFF73BFC124B1A689A4298
:1016B00004D0996993688A689A420BD3002383F314
:1016C000118894F8213003F00303012B06D0022B7C
:1016D00009D010BD0848FFF7C3FBEFE7E069BDE89C
:1016E000104000F0CDBA206CE169BDE8104000F078
:1016F0004FBB00BFD888FF1FD07900006C79000075
:1017000038B5124B9C69A36A606204F128059D42BA
:1017100007D01A68A2621846FFF712FDA36AAB420F
:10172000F7D194F8223043B994F821309B0704D1C3
:10173000636922691A61226953610F20FFF788FDEE
:101740000348BDE83840FFF78BBB00BFD888FF1FB8
:1017500060790000000000000000000000000000B0
:1017600010B52023044683F31188FFF7C9FB2046F8
:10177000BDE81040FFF7C4BF0000000000000000FB
:1017800010B52023044683F31188FFF7B9FB14B981
:101790000C48FFF765FB21460820FFF789FDFFF79E
:1017A000BFFB094B1A689A4207D0996993688A6807
:1017B0009A4202D20548FFF753FB002383F31188B6
:1017C00010BD00BF94790000D888FF1FD0790000B9
:1017D00070B50368074D0446AE6913B10648FFF7BC
:1017E0003FFB266003207462FFF732FDAB69586A45
:1017F00070BD00BFD888FF1FC07900000000000046
:1018000070B5046884B194F82030032B0E46054669
:1018100002D00648FFF724FB00232B6066622046B7
:10182000BDE87040FFF78CBC70BD00BF5079000070
:1018300069B1084B10B4024644689B69042083E8F0
:101840001400236053605DF8044BFFF731BD4FF087
:10185000FF307047D888FF1F000000000000000024
:1018600038B50468A04210D02368036094F82020A3
:101870005860042A0D4602D00448FFF7F1FA656269
:101880002046BDE83840FFF75BBC38BDA0790000BA
:1018900038B5202383F311880D4CFFF731FB256900
:1018A00095F82230013385F82230FFF739FB2368A1
:1018B000A34207D0A2699B6892689A4202D2054867
:1018C000FFF7CEFA002383F31188284638BD00BF06
:1018D000D888FF1FF479000000000000000000001D
:1018E00070B52023064683F31188FFF709FB144DDA
:1018F0003469AC4222D094F82230FF2B18D0013347
:1019000084F82230FFF70CFB2B680D4AAB4207D05E
:1019100092699B6892689A4202D20A48FFF7A0FA3D
:10192000002383F311883046FFF78AFE204670BDFE
:101930000548FFF795FA94F82230E0E70024E1E744
:10194000D888FF1FF4790000007A00000000000032
:1019500010B50446FFF79CFF034603E0FFF7C0FF06
:10196000034618B1DA69A2421846F7D1184610BDED
:1019700010B5044620B1002324606460A36010BD4C
:101980000148FFF76DFAF6E7107A0000000000004A
:101990003B4B70B505469C69FFF74AFB002D6BD0A9
:1019A000A868002836D0A26883689A4207D990F8C0
:1019B00020308260062B46D0072B30D0FBB12B465F
:1019C00003E09968A268914202D31B689D42F8D156
:1019D0005A6862602360062014605C606562FFF7ED
:1019E00037FCAB68A34202D02648FFF739FAA36B55
:1019F000AB4213D02348BDE87040FFF731BA90E8FE
:101A00000C00012180F820101A6002685360FFF773
:101A100097FBD4E7A36BEB60AC60A56370BD90E867
:101A20000A001960466A01684B60334602E0996813
:101A3000914202D31B689E42F9D15A68426003600A
:101A400010605860BBE790E80A001960466A0168B8
:101A50004B60334602E09968914202D31B689E4274
:101A6000F9D15A684260036010605860B068A2689B
:101A7000836893429BD3A2E70248FFF7F1F98FE70F
:101A8000D888FF1F207A000000000000000000003E
:101A900010B52023044683F31188FFF731FA20465E
:101AA000FFF776FFFFF73CFA074B1A689A4207D018
:101AB000996993688A689A4202D20448FFF7D0F97C
:101AC000002383F3118810BDD888FF1F387A0000E7
:101AD0002DE9F041DFF8C0800646D8F818700028DC
:101AE0004ED0202383F31188FFF70AFABB6B002B3B
:101AF0004AD09A68BA4203D02648FFF7B1F9BB6BC7
:101B00009E4202D02348FFF7ABF9F368BB63FFF7AF
:101B10008FFA33689E4230D0BC6BFD6B64B1FFF727
:101B200087FA23689C4203D09B689D4238BF1D46BC
:101B3000E468002CF3D133681A68996BBD601846CD
:101B400032605660B360F1609E63FFF7F9FAFFF709
:101B50005FFCFFF7E5F9D8F800300F4A434507D09E
:101B600092699B6892689A4202D20C48FFF778F912
:101B7000002383F31188BDE8F0810023B360E8E718
:101B80000448FFF76DF9ACE70248FFF769F9BB6B52
:101B9000AFE700BF2C7A0000D888FF1F387A00001A
:101BA0000349044B0448054A08601A60704700BFA7
:101BB0005889FF1F5489FF1F2894FF1F00800020B1
:101BC00038B50C460546FFF723FA14B1631E2342CD
:101BD00002D00A48FFF744F9094A0A4B10681B680B
:101BE00001386142013D204408402C440C401B1A3E
:101BF0009C429ABF24181460002038BD447A00002B
:101C00005889FF1F5489FF1F0000000000000000DA
:101C100038B505460C46202383F31188FFF770F989
:101C200021462846FFF7CCFF0446FFF779F9084B19
:101C30001A689A4207D0996993688A689A4202D2D0
:101C40000448FFF70DF9002383F31188204638BDBF
:101C5000D888FF1F587A0000000000000000000034
:101C6000044B054A1A6003F1100000229A60DA6002
:101C7000FFF77EBE6089FF1F111C000000000000FE
:101C80002DE9F041804698B310F0070F30D158F895
:101C9000043C58F8086C0733DB0806F1100748F8D5
:101CA000043C3846FFF7F4FE08363446A8F1080530
:101CB000AC4205D86368013304EBC3039D420CD3E7
:101CC000B4420FD0AC420DD32468AC42F8D863685C
:101CD000013304EBC3039D42F2D22048FFF7C0F862
:101CE000B442EFD123683BB19D4205D31C46DFE7E8
:101CF0001A48FFF7B5F8CAE758F8042C48F8083C2A
:101D00002560531C58F8080C05EBC30181420AD02A
:101D10006268531C04EBC3039D4213D03846BDE8F0
:101D2000F041FFF7D5BE496855F8333048F8083C14
:101D30005318013348F8043C6268531C04EBC30396
:101D40009D42EBD118E90A0013440133216063601E
:101D50003846BDE8F041FFF7BBBE00BF647A000023
:101D600038B504460D46FFF753F924B11DB1236879
:101D70002B60256038BD0348FFF772F823682B609D
:101D8000256038BD707A00000000000000000000EF
:101D900038B505460C46202383F31188FFF7B0F8C9
:101DA00028462146FFF7DCFFFFF7BAF8074B1A6811
:101DB0009A4207D0996993688A689A4202D2044885
:101DC000FFF74EF8002383F3118838BDD888FF1F32
:101DD0007C7A00000000000000000000000000000D
:101DE000EFF30983203383F30988002383F31188F9
:101DF000704700BF0000000000000000000000006D
:101E0000202383F311880F4B5B6813F4006302D126
:101E100083F31188704710B5EFF309844FF0807396
:101E200044F8043CA4F1200383F30988FFF7B0FAD7
:101E300018B1054B44F8083C10BD044B44F8083C6D
:101E400010BD00BF00ED00E01505000020050000FA
:101E500008B500F0D5FD054800F0FAFE00F058F98D
:101E600001F04EFBBDE8084000F002B8D47B000052
:101E700000F026BF0000000000000000000000008D
:101E80002DE9F041069F0D4690461E460446B8B126
:101E9000B1B1012A14D908F1040206FB0251002352
:101EA000A261079A616124606460A6602561E560B3
:101EB000E6612562E76222636362A362BDE8F081A6
:101EC0000148FEF7CDFFE6E7B87A00000000000009
:101ED00038B504460D46FFF79BF82369E2689A423D
:101EE00004D0184650F8043B2B6038BDA268002A85
:101EF000F7D0002038BD00BF000000000000000047
:101F000010B50446FFF784F8E36821698B4212D0CC
:101F1000A3696069A2680B448342236102F1010254
:101F200028BF236AA26028BF236120460021BDE8A4
:101F30001040FFF795BCA368002BE9D00248FEF7DC
:101F40008FFF2169E4E700BFD47A000000000000A1
:101F500038B504460D46FFF76BF803E0FFF768FC61
:101F600000280DDBA36820462946002BF6D0A36885
:101F70003BB1E268A369111D13446162A3620020B2
:101F800038BD0248FEF76CFFF3E700BF887A000017
:101F900070B50D460446FFF74BF8D5B1A369043B75
:101FA0009D4216D8A368D3B1E16860690D60A3694A
:101FB000A2680B448342E36024BF236AE360013AD2
:101FC000E36AA260002262626BB12046BDE8704005
:101FD00018470548FEF744FFA368002BE4D10248E8
:101FE000FEF73EFFE0E770BDA47A000000000000AD
:101FF00070B5202304460E46154683F31188FEF77C
:102000007FFF636AF3B11E70636AA26A0133934271
:10201000636211D2FEF784FF184B1A689A4207D008
:10202000996993688A689A4202D21548FEF718FFA8
:10203000002080F3118870BDA16920460439FFF7A4
:10204000A7FFE7E729462046FFF782FF054608B9C4
:10205000636AD8E7FEF764FF084B1A689A4207D014
:10206000996993688A689A4202D20548FEF7F8FE99
:10207000002383F31188284670BD00BFD888FF1F56
:10208000C87A00000000000000000000000000000E
:1020900010B50446FEF7BCFFE26823699A4201D0FE
:1020A000002010BDA368002BFAD0636A002BF7D084
:1020B000043B9B1AF4D01360A3696069A1681A44B9
:1020C000824228BF236AE26001F1FF3128BFE3604A
:1020D0000023A1606362012010BD00BF000000006A
:1020E00010B5044690F8D63080F8DE3001F070F874
:1020F00063681B6813B120460121984703232370AE
:1021000010BD00BF00000000000000000000000043
:1021100000F0EEBF00000000000000000000000022
:10212000012330B4002200F1840503702946426087
:1021300000F1480343F8042FAB424FF0000441F88C
:10214000042FF7D10481448130BC704700000000A7
:1021500038B50D46044668B361B3202383F3118874
:10216000FEF7CEFE2378013B012B02D91348FEF780
:1021700077FE656004F1080304F14801002243F88A
:10218000042F8B42FBD1204600F0CAFF02232370AC
:10219000FEF7C6FE0A4B1A689A4207D099699368FF
:1021A0008A689A4202D20748FEF75AFE002383F358
:1021B000118838BD0148FEF753FECEE7287B0000AA
:1021C000D888FF1F447B00000000000000000000D2
:1021D000F8B504460E461546FEF71AFF04B3FDB1E6
:1021E0002378042B02D01048FEF73AFE04EB860752
:1021F000FB6813B10C48FEF733FEFD60686918B147
:102200000021142205F094FAA86918B100211422C3
:1022100005F08EFA20463146BDE8F84000F0E8BFF0
:102220000148FEF71DFEDBE7507B000000000000C8
:102230002DE9F0418046FEF7EBFEB8F1000F3CD0EF
:1022400098F80030042B02D01E48FEF709FEB8F8BB
:102250000820B8F80A3002F0010203F00103A8F8E0
:102260000820A8F80A3008F10C0408F148062027D5
:10227000002554F8043FC3B187F31188FEF768FEC8
:102280002368586928B10C306FF00101FFF7B8FAE4
:1022900023689B696FF0010103F10C000BB1FFF79C
:1022A000AFFAFEF76DFE85F31188B4422560E0D1E8
:1022B0004046BDE8F04101F053B80248FEF7D0FDBA
:1022C000BEE700BF647B00000000000000000000CB
:1022D0002DE9F0410546884617461E46FEF798FE52
:1022E000F5B1B8F10F0F1BD8012404FA08F36A897D
:1022F0009CB2144203D00C48FEF7B2FD6A8905EB8C
:1023000088031443DB686C819B6900229F601E6018
:10231000284641465A60DA60BDE8F04101F090B8C5
:102320000148FEF79DFDDFE7EC7A000000000000A9
:102330002DE9F0410546884617461E46FEF768FE21
:10234000F5B1B8F10F0F1BD8012404FA08F32A895C
:102350009CB2144203D00C48FEF782FD2A8905EB9B
:1023600088031443DB682C815B6900229F601E6038
:10237000284641465A60DA60BDE8F04101F070B885
:102380000148FEF76DFDDFE7147B00000000000050
:102390002DE9F0470223002507460370A0F8DC5022
:1023A00080F8DE5080F8DF500581458100F1080497
:1023B00000F148064FF0200854F8043FC3B188F3F9
:1023C0001188FEF7C5FD2368586928B10C306FF0FD
:1023D0000101FFF715FA23689B696FF0010103F112
:1023E0000C000BB1FFF70CFAFEF7CAFD85F311885C
:1023F000B44225604FF00009DED187F8C49038461A
:1024000000F086FF7B681B6823B138464946BDE86B
:10241000F0471847BDE8F08700000000000000000A
:10242000F8B5436801781B6880F8E010052205467E
:1024300002700BB10421984705F1080420274835A4
:10244000002654F8043FC3B187F31188FEF780FDDE
:102450002368586928B10C306FF00101FFF7D0F9FB
:1024600023689B696FF0010103F10C000BB1FFF7CA
:10247000C7F9FEF785FD86F31188AC42E1D1F8BDBE
:10248000426890F8E010126801700AB10521104707
:10249000704700BF000000000000000000000000C6
:1024A000F8B50023044680F8C43000F1D40200F0EF
:1024B00097FF63689B684BB32046984730B3D4F8C6
:1024C000CC5094F8D43094F8DB1094F8DA2042EA37
:1024D0000122AA423CBFC4F8CC2015461B0600F1DD
:1024E0008D80002D74D1052384F8C430202383F31C
:1024F0001188FEF72DFD204629462A462B46FFF778
:1025000017FFFEF73DFD85F31188F8BD94F8D43030
:1025100013F0600711D02046002100F0B9FF2046DB
:10252000002100F0A5FF63681B6813B12046062157
:102530009847062384F8C430F8BD94F8D55003F0CA
:102540007F0242EA0526B6F5407F00F034811AD9B1
:10255000B6F5C06F00F013817AD9B6F5106F00F0B0
:10256000888040F60242964200F0FF80B6F5006F88
:10257000D1D104F1DF020125C4F8D070C4F8C8201D
:10258000C4F8CC509FE7022E00F0D28040F2C58004
:10259000B6F5807F00F08280B6F5817FBBD194F8DC
:1025A000D620002AB7D194F8D82012F00F0107D016
:1025B0001506204600F1218100F07AFF94F8D4300E
:1025C0000025C4F8C850C4F8CC50C4F8D0507AE7FD
:1025D000042384F8C430202383F31188FEF7B8FC69
:1025E000D4F8CC30D4F8C82020460021FFF770FE84
:1025F000FEF7C6FC002383F31188F8BDADB10123BB
:1026000084F8C430202383F31188FEF7A1FCD4F8AA
:10261000CC30D4F8C82020460021FFF789FEFEF711
:10262000AFFC002383F31188F8BD032384F8C43082
:10263000202383F31188FEF78BFC204629462A4687
:102640002B46FFF745FEFEF79BFC85F31188F8BD8E
:1026500040F20232964234D0B6F5A06F7FF45BAF01
:102660006B4AC4F8C870C4F8CC703D46C4F8D0209A
:1026700029E794F8D62094F8DF109142A0D023786F
:10268000042B32D072B3636884F8DF201B68042205
:1026900022703BB320460221984723E094F8D620CD
:1026A000012A7FF438AFB4F8DC20C4F8C87022F0F7
:1026B0000202C4F8CC70C4F8D0703D46A4F8DC2007
:1026C00001E794F8D620002A7FF425AF94F8D820AB
:1026D00012F00F013FF474AF1206204600F1928011
:1026E00000F0C6FE94F8D4306AE7202383F3118803
:1026F000FEF72EFC2046FFF79BFDFEF741FC87F31B
:102700001188636884F8DF701B68032121700BB1A6
:102710002046984794F8D620B4E71EBB04F1DC02AB
:102720000225C4F8D060C4F8C820C4F8CC50CAE66A
:1027300094F8D81011F0800F204601F00F014DD110
:1027400000F01EFE01284DD002287FF4E4AE314B8C
:10275000C4F8C830C4F8CC00C4F8D070054694F86A
:10276000D430B0E6012E7FF4D6AE2B4AC4F8C82090
:1027700002250022C4F8CC50C4F8D020A3E6626839
:1027800094F8D90094F8D830556894F8D71094F894
:10279000D62043EA00232046A84700283FF4BBAEDA
:1027A00043680568C4F8CC50C4F8C830C4F8D07089
:1027B00094F8D43087E694F8D620012A7FF4ABAEA3
:1027C000B4F8DC20C4F8C87042F00202C4F8CC703F
:1027D000C4F8D0703D46A4F8DC2074E600F0E8FDB3
:1027E0000128B1D10D4BC4F8C830C4F8CC60C4F88E
:1027F000D070354694F8D43065E600F069FE94F860
:10280000D430DDE600F044FE94F8D430D8E600BFC2
:10281000E1200000347B0000007B0000047B00000E
:1028200038B590F8C4300446062B47D8DFE803F0EB
:1028300004192A04043E07002C48FEF711FB204629
:10284000002100F025FE2046002100F011FE636803
:102850001B6813B1204606219847062384F8C4302C
:1028600038BD90F8DB1090F8DA30D0F8CC2043EA8D
:102870000123934206D9C3681D8AB2FBF5F305FB19
:10288000132505B3032384F8C430202383F3118870
:10289000FEF75EFB00210B4620460A46FFF718FDB7
:1028A000FEF76EFB002383F3118838BDD0F8D030DB
:1028B00003B19847002384F8C43038BD0B48BDE805
:1028C0003840FEF7CDBA202383F31188FEF740FB92
:1028D000204629462A462B46FFF72AFDFEF750FBE5
:1028E00085F31188022384F8C43038BD087B0000CA
:1028F00090F8C43010B50446062B3BD8DFE803F04F
:102900000404042D190407001D48FEF7A9FA204607
:10291000002100F0BDFD2046002100F0A9FD636804
:102920001B6813B1204606219847062384F8C4305B
:1029300010BD052380F8C430202383F31188FEF7EF
:1029400007FB00210B4620460A46FFF7F1FCFEF785
:1029500017FB002383F3118810BDC3689B695B6874
:102960003BB9D0F8D03003B19847002384F8C43085
:1029700010BD10BD0248BDE81040FEF771BA00BF9F
:10298000387B000000000000000000000000000094
:1029900043099B0010B403F1604300F1604404F567
:1029A000614403F56143090100F01F0001228240E8
:1029B000C9B284F80013C3F880211A605DF8044B93
:1029C000704700BF00000000000000000000000091
:1029D0000B2838B504460D4602D90548FEF740FAE3
:1029E00004F1604000F56D402D01EDB2057638BD73
:1029F0007C7B0000000000000000000000000000E0
:102A0000704700BF00000000000000000000000050
:102A10002DE9F0433C4E3D4DDFF8F8803C4FDFF8A8
:102A2000FCE0DFF8FCC04CF220524DF62813F28196
:102A3000F381348824F001042404240C41F2380981
:102A40000FCD348058F8096089B06C4646F478564A
:102A500048F809600FC495E80F0084E80F000023D0
:102A600084220A21CEF84830CEF84C308CF8001081
:102A70007A707A7842F020027A70ADF1040252F84E
:102A8000041FB1F5007FD8B203F1010335D0082B44
:102A9000F5D1B8231E4A137093799907FCD51C4AC7
:102AA0009379DB06FCD41A498B79194A03F00C039D
:102AB000082BF9D1072158231171114653718B79D5
:102AC000134A03F06003602BF9D1124B124F41F20D
:102AD000440141F2480641F2040400204FF48035DD
:102AE0005F50985111461D5110708B7903F00C0303
:102AF0000C2BFAD109B0BDE8F083C30003F0380312
:102B000043F08003C6E700BF00200540CC770000FB
:102B10000040064000700440000003110090044093
:102B2000005006400000000000000000000000000F
:102B30000069C84000F00100704700BF00000000BD
:102B40001F2970B50E46044615462CD8626901232C
:102B5000B340062D0CBF134322EA03036361344BD9
:102B60009C425CD040339C425BD040339C425AD064
:102B700040339C4259D040339C424ED02D48FEF702
:102B80006FF90023162D0DD8DFE805F0112511206F
:102B90001B2511160C0C0C0C0C0C0C0C11423D38A6
:102BA000332E290070BD2348FEF75AF9CEE74FF4C3
:102BB000807243F8262070BD4FF4907243F82620AF
:102BC00070BD4FF4817243F8262070BD40F20312AD
:102BD00043F8262070BD002243F8262070BD4FF434
:102BE000E06243F8262070BD4FF4C06243F826200F
:102BF00070BD4FF4A06243F8262070BD4FF4806290
:102C000043F8262070BD4FF4407243F8262070BD73
:102C10004FF4007243F8262070BD074BB2E7074B14
:102C2000B0E7074BAEE7074BACE7074BAAE700BF9F
:102C300000F00F409C7B000000D004400090044056
:102C400000A0044000B0044000C0044000000000A8
:102C50000C4941F23802F8B58B5843F478538B5045
:102C6000064600F5257735460024E1B2306855F870
:102C7000042F0134FFF764FF202CF6D18436BE42C6
:102C8000F1D1F8BD00700440000000000000000019
:102C900008B5FEF78DF9202383F31188FEF758F964
:102CA000FEF7E6F8FEF76CF9002383F31188FEF7D0
:102CB00097F9BDE80840FFF7A3B800BF0000000087
:102CC000054B4BF67F3000210722586099600B209E
:102CD00008211A60FFF77CBE10E000E00000000051
:102CE00000EB8100F0B4C368134F5D691B8A287C38
:102CF0009A4228BF1A4640F0020343EA810152B1CA
:102D0000002307EBC106AC687068E45CC45401336F
:102D10009342F8D1287C6C7CA30143F0880384F0B3
:102D2000010480F0010043EA024247F83120287490
:102D30006C74F0BC704700BF0090FF1F00000000E3
:102D4000F0B500EB8100DFF86CE0D0F80CC0BCF807
:102D50001230DCF818609A42B47C28BF1A4644EA64
:102D6000810122B300230EEBC1077D68B468ED5CDE
:102D7000E55401339342F8D1BCF81240F27C930140
:102D800043F0880343EA04434EF8313082F00102F5
:102D9000F274C1688A69136833B1498A013B0B44F4
:102DA000B3FBF1F31382F0BD01231382F0BD1C4687
:102DB000E4E700BF0090FF1F0000000000000000DB
:102DC0002DE9F84FC64B93F88040E4B2FEF7F0F8D7
:102DD00063070BD5DFF80C83D8F80430DB680BB140
:102DE00040469847BE4B042283F88020270740F1D5
:102DF000F480DFF8F082DFF8F0A2B94D4FF0010B5C
:102E00000DE00D2B00F0CE80012B68D0082385F853
:102E1000803095F88040E4B2260740F1DE8095F8D6
:102E20009030DBB21E09B71CC3F3800208EB8700A9
:102E3000B100C3F3C00341EA0204D0F8049044EAAD
:102E400043042BB9D9F81830002B00F0A1809A74F4
:102E50005AF83420C2F38303092BD2D1D9F81430A5
:102E6000002BD3D04EB998F8D41098F8D52042EA68
:102E70000122B2F5A06F00F0EC8093E806005AF84A
:102E80003400C0F3094002448A425A60C0F0C68050
:102E9000D9F80830002BB9D008EB8703B8F8082020
:102EA00059680BFA06F38C6822EA0303A8F8083085
:102EB00014B131468B48A047202383F3118808EBD7
:102EC0008707FEF745F87B68586900210C30FEF74C
:102ED00097FCFEF755F8002383F3118896E7D9F89D
:102EE0001830002B92D0C2F30944202383F31188B9
:102EF000FEF72EF8314622467A48FFF721FFFEF70B
:102F00003FF8002383F31188002C3FF47FAFD9F8FA
:102F10001800B9F812C0B0F810E081684268036880
:102F20000EF1FF3E214422441B1B1FFA8EFEA445D6
:102F3000816042600360A0F810E040F28580D9F81B
:102F40000C30002B3FF462AF08EB8703B8F80A207F
:102F500059680BFA06F3CC6822EA0303A8F80A3092
:102F600014B131465F48A047202383F3118808EB52
:102F70008707FDF7EDFF7B689B6903F10C0059683B
:102F8000FEF73EFCFDF7FCFF002383F311883DE7CD
:102F90005AF83430C3F38303092B3FF45FAF0D2B92
:102FA0007FF434AFB8F80A30D9F81470D9F8044077
:102FB0004C4841F0020E41F0030C002223F00103C3
:102FC0004AF83E2031464AF83C20A8F80A3087F8F3
:102FD00011B0A04785F894B018E7E50768D420063B
:102FE00061D4A10708D53E4B93F888200221D2B2C4
:102FF00083F8882083F88010E20607D539480378E3
:10300000042B62D0364B102283F88020A30637D4DD
:10301000FDF7E6FFBDE8F84FFEF7F2BE9A681044F0
:103020009860202383F31188FDF792FFD9F81430BC
:103030002C480CCB3146D21AFFF752FEFDF7A0FF09
:10304000002383F31188E1E6BEF1000F7FF4DEAECA
:1030500075E7244B234A93F8D6302249526881F809
:10306000DE3003F07F0385F89830136813B108460B
:1030700001219847032388F80030D9F81430FCE682
:10308000174C184894F8843003F0DF0384F8843038
:10309000FFF7F6F9202384F88030FDF7A1FFBDE8A3
:1030A000F84FFEF7ADBE0E4B802283F8802098E7E4
:1030B0000C48FFF76DF90A4B012283F88020FDF7D9
:1030C0008FFFBDE8F84FFEF79BBEFFF7A9F9044A52
:1030D00092F8843043F0200382F8843092E700BFF6
:1030E000002007409489FF1F0090FF1F0000000090
:1030F00010B50748FFF714F8064B41F2040141F2FE
:1031000048005A58022442F480225A501C5010BDE4
:103110009489FF1F007004400000000000000000C0
:103120000378012B00D07047254B9842FBD1002338
:10313000244A194602EBC30042F833100133102B26
:103140004160F7D130B4204D204B41F23404184691
:10315000295941F48021295193F80C1141F0800143
:1031600083F80C1190F80C11184B0906FAD4FF21C2
:10317000C2F30724C2F30740120E83F89C4083F881
:10318000B00083F8B42083F8801083F88810197495
:1031900093F80C21032042F04002002183F80C2117
:1031A00083F8940083F8001193F8842042F0010220
:1031B00083F884204920022130BCFFF7E9BB00BF1F
:1031C0009489FF1F0090FF1F0070044000200740FB
:1031D00090F8DE30024A03F07F0382F8983070479F
:1031E0000020074000000000000000000000000078
:1031F000102962D800EB81032DE9F041DD68AB694D
:103200008BB36C8A3E4A3F4824048E00002744F06A
:10321000880E9F74DF7442F836E003783F2B4DD858
:103220000378394FDBB203F1010C46F0010602EBE3
:10323000411E07EB831344F0C8045FFA8CFC80F84E
:1032400000C0CEF8043042F8364003783F2B36D821
:103250000378DBB202EBC6025E1C07EB8314F3B209
:103260000370082354606C69002C36D04FEA810E3D
:103270004EF00206224A23484FF0000C84F810C09A
:1032800084F811C042F836C004783F2C37D804784F
:103290001D4FE4B204F1010802EBC6064EF0030E26
:1032A00007EB84145FFA88F880F80080746042F8B5
:1032B0003EC004783F2C03D9FEE77047FEE7FEE7E7
:1032C0000478E4B2661C02EBCE0243F0040307EB81
:1032D0008414F6B20670DBB254602A6802F003026E
:1032E000012A03D043F00103DBB212B143F0100313
:1032F000DBB23031054A02F82130BDE8F081FEE74B
:103300000090FF1F0092FF1F7C8AFF1F00200740D4
:1033100070B50F490F4C104B002502220D70064668
:1033200084F894202946C360FFF762FFFF239F21A2
:10333000012284F8883084F8803086F8DE5084F8E2
:10334000985084F88C3084F8841084F8942070BDF0
:103350000092FF1F00200740B07B0000000000002B
:1033600005480123002103F130020133102B00F83E
:103370002210F8D1704700BF002007400000000075
:103380000F2913D8890001F1804101F5E42191F85A
:10339000C03003F0080303F0FF0043B191F8C030E0
:1033A00013F0020F14BF0120022070470020704765
:1033B0000F2913D8890001F1804101F5E42191F82A
:1033C000C03003F0040303F0FF0043B191F8C030B4
:1033D00013F0020F14BF0120022070470020704735
:1033E000F0B500EB8100144DC3689F6997F812E0B7
:1033F000890041EA0E0E013A05EBCE0500236C6808
:103400000D4EE45C02F8014F0133082BF7D1C2687E
:10341000BB7C528A120442F0880246F83E20C26801
:10342000528A83F001031204194342F0C8030122B7
:1034300046F83130FA74F0BD0090FF1F0000000024
:1034400000EB8101C9688A69136833B1498A013B7D
:103450000B44B3FBF1F313827047012313827047CF
:1034600000EB8103DB685B691A68FFF739BC00BFBA
:10347000890001F1804101F5E42191F8C03043F069
:10348000020381F8C0307047000000000000000017
:10349000890001F1804101F5E42191F8C03043F049
:1034A000020381F8C03070470000000000000000F7
:1034B000890001F1804101F5E42191F8C03003F069
:1034C000FD0381F8C03070470000000000000000DC
:1034D000890001F1804101F5E42191F8C03003F049
:1034E000FD0381F8C03070470000000000000000BC
:1034F000FFF78EBA0000000000000000000000008E
:10350000704700BF00000000000000000000000045
:103510000139212912D8DFE801F01A2923111111EC
:10352000111111111111111111111111111111118B
:10353000111111111111111111111C1300207047DB
:10354000042BFBD8DFE803F0141C1A1816001248ED
:103550007047042BF4D8DFE803F015191D1B170082
:10356000032AEBD80D4B03EBC20070470C487047A1
:103570000C4870470C4870470C4870470C4870471F
:103580000C4870470C4870470C4870470C4870470F
:103590000C4870470C487047E07E0000EC8000004B
:1035A000007F0000D87E0000B08100009481000000
:1035B000F87E00000C8100009C810000687E000005
:1035C0005C800000947E0000548100000000000038
:1035D000704700BF00000000000000000000000075
:1035E000704700BF00000000000000000000000065
:1035F000704700BF00000000000000000000000055
:10360000704700BF00000000000000000000000044
:10361000704700BF00000000000000000000000034
:1036200010B5046B2378042B82B001D002B010BD1A
:1036300023891B07FAD4064801A9FEF749FC024674
:103640000028F3D0204603211023FEF771FEEDE79A
:10365000FC92FF1F000000000000000000000000BE
:1036600010B5202382B0044683F31188FDF770FC67
:10367000FDF7CEFC1248C3680BB1FDF729FD2346C8
:103680000F48104A3221FDF7F3FCA3695B691B6800
:103690008BB90D4801A9FEF71BFC024620B120465C
:1036A00003211023FEF744FEFDF76AFC002383F399
:1036B000118802B010BD0448FEF722FCE9E700BF04
:1036C0007092FF1F61370000FC92FF1F0000000096
:1036D00038B50446202383F31188FDF739FC23789D
:1036E000042B20D1174B1B78EBB9174D2A78D2B198
:1036F00023899B071DD54FF47A7303FB02F3134D07
:1037000003F2E733A5FB0335FDF782FC1048C368DD
:10371000AD09AD000BB1FDF7DBFC294623460C4893
:103720000C4AFDF7A5FCFDF72BFC002383F3118861
:1037300038BD094A204601210823FEF7F9FD2A7801
:10374000D9E700BF3186FF1FF092FF1FD34D6210F3
:10375000DC92FF1FD13600003093FF1F00000000F5
:1037600010B5202384B0044683F31188FDF7F0FBE5
:103770002378042B06D123891B0703D41A48FEF7AC
:1037800087FC98B9FDF744FC1848C3680BB1FDF7F6
:103790009FFC23461548164A3221FDF769FCFDF7C8
:1037A000EFFB002383F3118804B010BD0E4803A97A
:1037B000FEF78EFB024680B1039B0F2B07D8134404
:1037C00002F11000002103F8011B8342FBD12046C7
:1037D00003211023FEF7ACFDD4E701900548FDF767
:1037E0003FFB019AE8E700BFFC92FF1F7092FF1FAA
:1037F0006137000080810000000000000000000030
:1038000038B590F8D43003F07F02212A044607D05F
:10381000B4F8D42040F281639A4232D0002038BDFF
:1038200023F07F0303F0FF029BB1002AF0D090F851
:10383000D530022B00F09C80032B57D0012BE7D111
:1038400090F8D830042B48D8DFE803F07C7E715D17
:103850007C0090F8D5300A2B00F081800B2B2BD008
:10386000092BD5D190F8D8300BB1042BD0D1594BBE
:10387000C4F8C83001200023C4F8CC00C4F8D0300C
:1038800038BD626894F8D90094F8D830556894F837
:10389000D71094F8D62043EA00232046A8470028F2
:1038A000BCD090E80C00C4F8C8300023C4F8CC2089
:1038B000C4F8D030012038BDB0F8D8306BB990F8DA
:1038C000D6304549454A003318BF01230B701370A9
:1038D0001BB9434D2B78002B4CD10023C4F8C830C2
:1038E000C4F8CC30C4F8D030012038BDB0F8D8309E
:1038F000002B8DD1C0F8D030374AC4F8C820012041
:10390000C4F8CC0038BD90F8D700012886D194F8CF
:10391000D630022B52D0032B80D1324AC4F8CC309F
:1039200000211370C4F8C820C4F8D01038BD2E4B45
:10393000C4F8C83010220023C4F8CC20C4F8D0301A
:10394000012038BD294BF3E7294BC0F8C8300522C8
:103950000023C0F8CC20C0F8D030012038BD1F4B68
:103960001F4D1A7890F8D7302B70002AB3D0B4E7E7
:103970001B4B7DE7202383F31188FDF7E9FA2A78B2
:103980001C4D4FF47A7303FB02F303F2E733A5FBFC
:103990000335FDF73DFB1848C368AD09AD000BB119
:1039A000FDF796FB234629461348144AFDF760FBB2
:1039B000FDF7E6FA002383F311888EE7094AC4F87D
:1039C000C820032500211370C4F8CC50C4F8D010CF
:1039D00038BD00BFD892FF1F0086FF1F3186FF1F32
:1039E000F092FF1F9892FF1F2092FF1F3093FF1F3E
:1039F000F492FF1FD34D6210DC92FF1FD1360000FE
:103A000008B503F085FE00F0BBFCBDE8084000F0FF
:103A100097BC00BF00000000000000000000000094
:103A200003F06EBE00000000000000000000000077
:103A3000042938B50C462ED0052927D0022900D0FC
:103A400038BD0546202383F31188FDF781FA284607
:103A50000121124AFEF7BCFB28462146104AFEF718
:103A6000B7FB284603210F4AFEF7B2FB2846042184
:103A70000D4AFEF7ADFB284605210C4AFEF7A8FBD0
:103A8000FDF77EFA002383F3118838BD02F0E8F8D1
:103A9000FFF7B6FF38BDFFF7C3FF38BDC880000091
:103AA000B07F0000A4800000087F00005C8100005F
:103AB000F0B5174A41F2340383B0D3585B0305468F
:103AC00007D502F52C3292F8083103F0EF0382F8A3
:103AD000083140F2DC50FDF753FE28460D490E4EEA
:103AE0000E4FFEF735FB0E4A0E4892F808310E498C
:103AF00043F0100382F8083100240195009710224A
:103B00000423F460FEF7BCF9084BDC6003B0F0BDA1
:103B100000700440E87E0000DC92FF1F21360000A8
:103B200000200740FC92FF1F2092FF1F7092FF1F92
:103B300010B5084C94F8943043F0040384F89430A2
:103B40000F20FDF71DFE94F8943003F0FB0384F87A
:103B5000943010BD0020074000000000000000006D
:103B6000014B1878704700BFD892FF1F000000007B
:103B700070B52023044683F31188384DFDF7C0F952
:103B80002B78042B15D0FDF7CBF9354B1A689A42E8
:103B900004D0996993688A689A4203D3002383F317
:103BA000118870BD2F48FDF75BF9002383F311885E
:103BB00070BD2B4EFDF7B4F93368B34207D0B2693C
:103BC0009B6892689A4202D22648FDF749F9002381
:103BD00083F31188244B1B7833BB202383F3118894
:103BE000FDF78EF92B891D4A9B072BD41B48012119
:103BF00022460823FEF79CFBFDF792F93368184A2A
:103C0000B34207D092699B6892689A4202D21548E3
:103C1000FDF726F9002383F31188144D20686168AD
:103C2000A268E3680FC570BD202383F31188FDF7F8
:103C300067F92B89094A99060AD4084805212246C2
:103C40001023D7E7136958690C30FDF7C1FDCDE7A4
:103C5000136A58690C30FDF7BBFDEEE79489FF1F2E
:103C6000D888FF1F488100003186FF1F3093FF1F57
:103C700038B50546202383F31188FDF741F9204B21
:103C80001B78042B0ED0FDF74BF91E4B1A689A4295
:103C900004D0996993688A689A422AD3002383F3EF
:103CA000118838BD174CFDF73BF92368A34207D0B4
:103CB000A2699B6892689A4202D21348FDF7D0F835
:103CC000002383F31188202383F31188FDF718F96B
:103CD0002A4605230A480221FEF72AFBFDF720F9B0
:103CE0002368084AA342D9D092699B6892689A4295
:103CF000D4D20548FDF7B4F8002383F3118838BD0A
:103D00009489FF1FD888FF1F488100000000000031
:103D100030B5202383B0044683F31188FDF7F0F813
:103D20000F480178042908D1022501AA0323ADF820
:103D300005408DF80450FEF7FBFAFDF7F1F8094B4A
:103D40001A689A4207D0996993688A689A4202D29F
:103D50000548FDF785F8002383F3118803B030BDD3
:103D60009489FF1FD888FF1F4881000000000000D1
:103D700030B5202383B0044683F31188FDF7C0F8E3
:103D80000F480178042908D103252B4601AAADF874
:103D900005408DF80450FEF7CBFAFDF7C1F8094B4A
:103DA0001A689A4207D0996993688A689A4202D23F
:103DB0000548FDF755F8002383F3118803B030BDA3
:103DC0009489FF1FD888FF1F488100000000000071
:103DD00010B52023044683F31188FDF791F8184BA2
:103DE0001B78042B13D0FDF79BF8164B1A689A42E8
:103DF00004D0996993688A689A4204D3002080F3BA
:103E0000118840B210BD1048FDF72AF8F6E7FDF71B
:103E100087F80C4B1A689A4207D0996993688A68A8
:103E20009A4202D20848FDF71BF8002383F3118859
:103E3000012221460548FEF7DBF8C0B240B210BDB2
:103E40009489FF1FD888FF1F48810000FC92FF1F44
:103E50000846FFF7BDBF00BF0000000000000000E3
:103E6000704700BF000000000000000000000000DC
:103E7000704700BF000000000000000000000000CC
:103E800010B5084C01F0BCFEB4F8DC309B0700D440
:103E900010BD01F0CDFE0028FAD02046BDE810404C
:103EA000FFF746BE9489FF1F0000000000000000DD
:103EB0001F4C08B5FDF7CCFFFCF782FFFFF7D0FFE2
:103EC0002046FFF7F5FD00201A4902F079F8237823
:103ED000042B05D03220FDF753FC2378042BF9D1B5
:103EE0003220FDF74DFC1448114D02F079F800F036
:103EF000AFFA124800F03CFA03F0DAFB104802F087
:103F00006FF8FFF7B5FF2378052B0ED10D4802F0AF
:103F100067F82B78052B04D1FFF7B2FF2378052B28
:103F2000FAD001F09DFB02F053FD00F0A1FAEAE7A0
:103F30009489FF1F513E0000B88100001C86FF1FBE
:103F4000CC810000E08100000000000000000000C3
:103F500070B5194C194E1A4D204603210222FEF766
:103F6000EFFD022120460A46FEF7EAFD2046042125
:103F70000222FEF7E5FD204607210222FEF7E0FDC2
:103F800030460D210222FEF7DBFD30460C210222D5
:103F9000FEF7D6FD204600210222FEF7D1FD28467D
:103FA00011210222FEF7CCFD284610210222BDE895
:103FB0007040FEF7C5BD00BFC0F00F4000F00F40DD
:103FC00040F00F4000000000000000000000000072
:103FD00038B5FFF7BDFF03210A462248FEF7B0FDC2
:103FE000204804210322FEF7ABFD1E4800210322D6
:103FF000FEF7A6FD1C4800210322FEF7A1FD0321C8
:104000000A461948FEF79CFD174802210322FEF7D5
:1040100097FD164805210322FEF792FD134806215D
:104020000322FEF78DFD0F4801210322FEF788FDD4
:104030000F4B104903F11200002223F8022F834294
:1040400021F8022FF9D10C4A064C1378202543F0B1
:10405000020313704FF4FA706560FDF791FBA560E1
:1040600038BD00BF80F00F4040F00F40C0F00F405F
:104070005293FF1F6693FF1F0494FF1F0000000070
:104080002DE9F04F8A4E8B4FDFF82CA2DFF83092EB
:10409000DFF8288283B035460024E3B2013B072BCA
:1040A00000F2B580DFE813F0AA00A100C800BC0050
:1040B000D10098000800F2007F4811210622FEF787
:1040C0003FFD4FF40033CAF808302023C8F80C3005
:1040D00003217A48FEF72CFD042110F1FF3B7748BD
:1040E00018BF4FF0010BFEF723FD01280CBF002382
:1040F00002230021714843EA0B0BFEF719FD01284A
:104100000CBF0023042300216B484BEA030BFEF78E
:104110000FFD01280CBF00230823032166484BEA4A
:10412000030BFEF705FD01280CBF0023102302211D
:1041300061484BEA030BFEF7FBFC01280CBF002390
:10414000202305215E484BEA030BFEF7F1FC012812
:104150000CBF00234023062159484BEA030BFEF70E
:10416000E7FC01280CBF00238023544801214BEABF
:10417000030BFEF7DDFC01280CBF00234FF4807316
:1041800035F8022F4BEA03039A420BD03A782B8082
:10419000484B2AB1DFF840B19BF80020D10760D42A
:1041A00005233B700134FFF7D3FE092C7FF475AF74
:1041B0003B78404A63B1013BDBB21370002B6FD1F7
:1041C000404B414936F8022F23F8022F8E42F9D195
:1041D000012003B0BDE8F08F394800210622FEF728
:1041E000AFFC0123C9F808306FE7354804210622E7
:1041F000FEF7A6FC1023C9F8083066E73048022114
:104200000622FEF79DFC0423C9F808305DE72C4820
:1042100003210622FEF794FC0823C9F8083054E76E
:10422000DFF8B8B00D2158460622FEF789FC4FF49E
:104230000053CBF8083048E7214807210622FEF753
:104240007FFC8023C9F808303FE7DFF890B00C21ED
:1042500058460622FEF774FC4FF48053CBF8083022
:1042600033E71A48019301F0BBFE9BF80020D20708
:1042700096D5019B1648197801F0B2FE9BF80030E4
:10428000DB078DD5134801F0ABFE89E70A48102102
:104290000622FEF755FC4FF48033CAF8083014E7C5
:1042A0000120FDF76DFA012003B0BDE8F08F00BFDB
:1042B0006693FF1F3086FF1F40F00F4080F00F40D5
:1042C000C0F00F405293FF1F7893FF1F8C820000B5
:1042D00098820000C48900000494FF1F00F00F4082
:1042E000014B33F8100070475493FF1F000000008B
:1042F00038B50D480D4D01F073FE002421460C48E1
:1043000001F06EFE0B4801F06BFE35F8020F01F074
:1043100017FC0146084801F063FE0134074801F02C
:104320005FFE092CEAD138BDA08200005293FF1F26
:1043300098820000FC890000B8820000C489000057
:10434000830704D4074805210222FEF7F9BB10B504
:10435000044C052120460622FEF7F2FB2023636071
:1043600010BD00BF80F00F40000000000000000002
:10437000014B1860704700BF8093FF1F00000000D2
:10438000024B186808B10368184770478093FF1FF5
:10439000154B1B68D3B170B5144E5B680446984743
:1043A00033785A0709D513F0010315D104F110052C
:1043B00023B90134AC42FBD14BB970BD0C48217814
:1043C00001F00EFE337803F00103F2E7704709486D
:1043D000BDE8704001F004BE074801F001FE3378EB
:1043E00003F00103E2E700BF8093FF1F0494FF1F67
:1043F000D4820000C4890000C082000000000000D8
:10440000024B1B680BB19B68184770478093FF1FD6
:10441000054B1988814205D0044918800B680BB1FF
:10442000DB681847704700BF7C93FF1F8093FF1F16
:10443000054B1988814205D0044918800B680BB1DF
:104440001B691847704700BF7A93FF1F8093FF1FB7
:1044500008B501F0DDFDFFF7BBFDBDE8084001F048
:10446000A7BE00BF00000000000000000000000028
:104470002DE9F04184B0FFF703FE3D4D3D4F4FF075
:1044800000085FFA88F63046FFF72AFF35F8024F3A
:104490004440A4B25CB13B78990721D4002344FA8C
:1044A00003F2D207D9B220D40133092BF7D108F196
:1044B0000108B8F1090FE4D1FF2300228DF808307C
:1044C0008DF809308DF80A2001F0AAFD40F00100B6
:1044D000ADF80C0004AB13E9030000F061F825E02F
:1044E0000190FFF705FF0198D8E701249C400442A2
:1044F00014BF012300238DF80A308DF808108DF8C1
:10450000096001F08DFD40F00100ADF80C0002AD36
:1045100095E8030000F044F895E8030001F048FB3B
:10452000154A32F818305C4022F81840134C01F05C
:1045300037FB02F0B5FAFFF723FF237883420DD053
:10454000FFF71EFF0B4B20701B785A0701D5DB07C6
:1045500007D404B0BDE8F04101F042BB04B0BDE8AF
:10456000F0810146064801F03BFD2078F1E700BFED
:104570008693FF1F0494FF1F8893FF1F8493FF1FE0
:10458000DC820000000000000000000000000000CD
:10459000FFF7D6BE00000000000000000000000091
:1045A000F0B587B08DE80300BDF804509DF80070A9
:1045B0009DF801606C466DB18DF808708DF809604A
:1045C000BDF808204FF6FF739A4203D09DE8030020
:1045D00001F0EEFA8DF800708DF80160ADF804502E
:1045E00094E80300002305930490ADF8141006AB83
:1045F00013E9030000F014FE07B0F0BD0000000056
:10460000F8B1822810B5044665D0832853D0842899
:1046100071D0031FDBB2A02B52D900F12003DBB213
:10462000072B78D900F15B03DBB2022B0AD8A5284F
:104630007ED0A6280CBF82208320BDE81040FFF763
:10464000E7BE704700F15803DBB2142B37D8A82817
:104650006CD0A9287AD0AA287AD0AB287AD0AC28F6
:104660007AD0AD287AD0AE287AD0AF287AD0B128C7
:104670007AD0B0287AD0B2287AD0B3287BD0B428A8
:104680007CD0B5287DD0B6287ED0B72800F08880B1
:10469000B82800F08280B9287CD0BA2877D0BB280F
:1046A00000F08180BC2840F22A2018BF0020BDE81D
:1046B0001040FFF7BDBEFFF763FEC2073AD510BD3D
:1046C00002F006FE0028FAD1204600F0F1FFBDE816
:1046D000104000F0C5BFFFF753FE8107EFD439202B
:1046E00000F0E6FF00F0BCFF392001F029F8BDE83A
:1046F000104000F0B5BFFFF743FE4307DFD447206B
:1047000000F0D6FF00F0ACFF472001F019F8BDE83B
:10471000104000F0A5BF00F007040120A040C0B287
:1047200001F066F8BDE8104000F09ABFE220BEE755
:10473000812082E7532000F0BBFF00F091FF53205F
:1047400000F0FEFFBDE8104000F08ABFE920AEE7B0
:10475000EA20ACE7B520AAE7B620A8E7B320A6E791
:10476000B420A4E7B720A2E7CC20A0E7CD209EE7A5
:1047700040F283109BE74FF4C57098E74FF4C9707F
:1047800095E74FF4CA7092E740F221208FE740F29C
:1047900026208CE740F2252089E74FF4097086E750
:1047A00040F2232083E740F2272080E7000000004A
:1047B000D0B1822808B503462CD0832815D0842890
:1047C0004ED0021FD2B2A02A34D900F12002D2B2B8
:1047D000072A3AD900F15B02D2B2022A15D958331E
:1047E000DBB2142B2CD908BD7047FFF7C9FDC207F7
:1047F000F9D5532000F05CFF00F032FF532000F0A9
:104800009FFFBDE8084000F02BBF0020BDE8084036
:10481000FFF7FEBDFFF7B4FD8107E4D5392000F0B6
:1048200047FF00F01DFF392000F08AFFBDE8084077
:1048300000F016BF00F084FFBDE8084000F010BF94
:104840000020BDE80840FFF7F3BD00F0070301209A
:104850009840C0B200F0D4FFBDE8084000F000BFAF
:10486000FFF78EFD4307BED5472000F021FF00F083
:10487000F7FE472000F064FFBDE8084000F0F0BEFE
:104880002DE9F04103468179828800689F7884B0E1
:104890000D09009059781878A2B38DF808008DF8AA
:1048A0000910BDF808404FF6FF7294422AD08DF8E7
:1048B00001108DF8000000981C4600F0A9FE064685
:1048C00000F09EFE00F0CCFDC6F303330F2B19D889
:1048D000DFE803F026263B3B617218187D18A4A47C
:1048E0001B1818B6002F00F05C81002D00F020810D
:1048F000A379D90724D56FF30713A371B8F1000F7B
:1049000040F01A8104B0BDE8F0812046F1B2C6F350
:10491000032201F055F804B0BDE8F04100F008BDF5
:10492000C6F3072303F0F003002B40F0F080C6F33A
:104930000324002F00F00881002C40F01281F0B217
:1049400004B0BDE8F041FFF75BBEC6F3072303F0F8
:10495000F003202B18BF4FEA1618F0B20CBFC6F3B5
:10496000032808F0F008002800F0DE800128B9D103
:10497000002F00F00E81052DC4D800F031FF10EAA1
:10498000080F00F0D580404600F03AFF04B0BDE8C3
:10499000F04100F065BEC6F38123002B00F0BB8020
:1049A000012BAFD1002F00F0F280C6F3090004B054
:1049B000BDE8F041FFF73CBDF0B2002F00F0A4804D
:1049C00001F0CEFE04B0BDE8F04102F001B816F4EB
:1049D000407F74D1002F95D1F2064FEAD60348BF2D
:1049E0000F2003F01C0306F00F0448BF9840C6F3E5
:1049F00081264CBFC0433846022E04FA03F400F06F
:104A00000081032E00F0DE80012E40EA040000F059
:104A1000DC8004B0BDE8F04100F04ABDF4B2A4F17E
:104A2000E003132B00F2A380DFE803F02E2E2E2EDE
:104A30002E2E2E2E2E2E2E2E2E2E2E2E3C251D13BD
:104A40002046F1B2C6F3032204B0BDE8F04100F005
:104A5000BFBF002F00F0C780C6F3042004B0BDE83C
:104A6000F04100F055BD47B1C6F3042004B0BDE8E5
:104A7000F04100F06DBD002FF6D0C6F3042004B065
:104A8000BDE8F04100F054BDC6F30420002F00F053
:104A9000AF8000F04DFD14F00F003FF433AF00F095
:104AA000A7FE73E7002F00F09A80042D3FF62AAF8F
:104AB000C6F3042004B0BDE8F04100F061BD002F52
:104AC0004CD0C6F30023002B3FF41CAFF20802F0D9
:104AD0001C0206F00F0406F01003944003F0FF00E0
:104AE00013B10F209040C043C6F38126022E00F080
:104AF0008E80032E5ED0012E40EA04005DD004B00B
:104B0000BDE8F04100F05CBD01F0B2FE5AE73409A7
:104B100004F0F0040DE7002F4AD0C6F3090004B0FA
:104B2000BDE8F041FFF774BC37B30DB1012D05D0DE
:104B3000B8F1000F3FF4E6AE4046B0E7404604B09F
:104B4000BDE8F04100F08CBEF0B2FFF731FE002C62
:104B50003FF4D8AE204600F073FE17E7C6F34023BB
:104B6000B1E7204600F064FE00F07AFDE7E68FB37F
:104B7000002D82D02046E3E615B1012D3FF4C2AEF0
:104B800000F076FEB8F1000F3FF4BCAEFBE638460D
:104B90000DE7042D3FF6B6AEB8F1000F3FF4B2AE0C
:104BA000F1E6002DF8D004B0BDE8F041FFF700BEFB
:104BB0003846B4E700F004FD204604B0BDE8F041FB
:104BC00000F0EEBC00F074FC204604B0BDE8F041FB
:104BD00000F05EBC002D3FF447AF2046E3E7052D13
:104BE0003FF690AE64E704B0BDE8F04100F080BC51
:104BF00000F0AEFC14F00F003FF484AE00F000FEB5
:104C0000C4E6204304B0BDE8F04100F061BC20439D
:104C100004B0BDE8F04100F0E3BC00BF00000000BC
:104C200008B500F015FE00F0CBFD00F019FD01F015
:104C3000EFFF01F0CDFE0020FFF7EAFB0020BDE80A
:104C40000840FFF7F5BB00BF0000000000000000B7
:104C500008B500F0E5FDBDE80840FFF7E1BF00BF83
:104C600000B583B0ADF80400019800F0D1FCC0F3AA
:104C70000333023B0D2B14D801229A4012F4105139
:104C800004D0C0F3C02003B05DF804FB40F203334E
:104C9000134053B1C3B2DF2B0BD9F02B09D0084618
:104CA000F1E7002003B05DF804FB184603B05DF89F
:104CB00004FB0120E7E700BF000000000000000047
:104CC00082B002AB03E9030002B0704700000000AD
:104CD00082B002AB03E9030002B07047000000009D
:104CE00070B50A4B0A4D1C782B78A3420CD0094EA4
:104CF00006EBC40393E80300FFF7EAFF01342B78C7
:104D000004F00704A342F3D170BD00BFE493FF1F7A
:104D1000E593FF1F9C93FF1F0000000000000000B0
:104D20002E498B791B0900D070478B78002BFBD064
:104D30002DE9F0472A4B2B4D1B782A789A4282B0F6
:104D400048D0DFF8A4C04FF6FF7EE04605E001330F
:104D50002A7803F007039A423CD08A880C78487876
:104D6000002AF4D08DF800408DF80100BDF80060F5
:104D70007645ECD0DF000CEB0706DFF86CA096F868
:104D800001908145E3D118F83300A042DFD1B0781B
:104D90000028DCD1B088824285BFC2F57F42FF3255
:104DA000821A1218C72ACCBF00220122002ACED0B4
:104DB00057448B79BA790948012464F3071264F3E4
:104DC0000713BA718B71FFF75BFD02B0BDE8F047C6
:104DD000FFF786BF02B0BDE8F08700BFDC93FF1F7E
:104DE000E493FF1FE593FF1F9C93FF1F000000004B
:104DF0002DE9F047C14D044696B0AB88006802909B
:104E000094F800E0627894F80290B4F8048028786E
:104E100069780DF1080C002B58D08DF810008DF832
:104E20001110BDF810704FF6FF76B74202D0AF7880
:104E3000002F60D18DF838008DF83910BDF838702A
:104E40004FF6FF76B74241D0AE78002E3ED14345B3
:104E500085BFC3F57F43FF33C3EB08034344C72B30
:104E6000CCBF00270127002F00F02A814F4687B3CF
:104E70008DF840008DF84110BDF840109F484FF666
:104E8000FF73994209D08DF808E08DF80920BDF82C
:104E900008100388994200F0E5808DF808E08DF84D
:104EA00009200298FFF7DCFE002800F0D38020687C
:104EB0006168924B03C3FFF733FF95E80300FFF7E8
:104EC00007FF0127384616B0BDE8F087B9F1000F9B
:104ED00007D12046FFF7D4FC0127384616B0BDE8BD
:104EE000F0878DF808E08DF809200298FFF7B8FEEA
:104EF0000028EED0DBE7434585BFC3F57F43FF3392
:104F0000C3EB08034344C72BCCBF00260126002E69
:104F100039D1AB79DFF8E4A113F0F00F00F0318163
:104F20008DF831108DF83000BDF830004FF6FF716C
:104F300088420AD08DF808E08DF80920BDF80800F5
:104F4000BAF80010884200F0A9808DF808E08DF8CA
:104F500009200298FFF784FE0028BAD0B9F1000FAB
:104F6000B7D0AB79654A1F2BA1D91288ADF8502074
:104F700014A80022ADF854808DF856308DF85220D8
:104F8000FFF77EFC93E795F806C05C4B1CF0F00F32
:104F90002BD18DF819108DF81800BDF818004FF6B8
:104FA000FF71884209D08DF808E08DF80920BDF81E
:104FB00008001988884200F015814F46B8F1000FAB
:104FC00079D08DF820E08DF82120BDF820104FF623
:104FD000FF7399426FD0B9F1000F00F08480AB7974
:104FE00043F00103AB71002777E78DF829108DF8A6
:104FF0002800BDF828004FF6FF71884209D08DF8CF
:1050000008E08DF80920BDF808001988884200F0F2
:10501000D1808DF808E08DF809200298FFF720FE76
:1050200000283FF456AFB9F1000F3FF452AFAB790F
:10503000324A1F2B7FF63BAF1288ADF8482012A8EA
:105040000022ADF84C808DF84E308DF84A20FFF7E5
:1050500017FC2CE7AB79204643F00103AB71FFF757
:105060000FFC3AE78379DA0700F1B7801A0900F0FC
:10507000B48019090F291A46A37103D0013161F3D5
:105080000712A2712046FFF7FBFB206861681B4BEB
:1050900003C395E80300FFF71BFE1EE7B9F1000FFD
:1050A0007FF453AFA3712046FFF7EAFBCAF80090E4
:1050B000CAF8049011E7B9F1000F3FF40EAF8EE784
:1050C0008DF808E08DF809208DF80A90ADF80C8075
:1050D0009CE80300FFF7F4FD2F606F6095E8030084
:1050E000FFF7F6FDF9E6064B06491B7891F80080BC
:1050F00043451DD0DFF810C0E1460BE0DC93FF1FF5
:10510000E493FF1FE593FF1F9C93FF1F05F0070328
:1051100043450DD00CEBC3015D1C48789042F5D19E
:1051200019F833307345F1D18B78002BEED0D4E6EB
:105130008DF809208DF808E0029800F069FAC0F3B4
:105140000333C2B2032B11D8DFE803F015150202B6
:1051500010F4706F04D0A37913F0F00F3FF4BDAEDC
:1051600002F12003DBB2072B7FF6B7AE2046FFF734
:1051700087FB3746B1E610F4706FF1D0002AEFD10B
:10518000ABE68DF808E08DF809208DF80A90ADF8AF
:105190000C809CE80300FFF793FD5046FFF770FB7F
:1051A000CAF80060CAF804609AE803003746FFF7BF
:1051B0008FFD92E6B9F1000F7FF42BAF204684F803
:1051C00006C00193FFF75CFB019B206861681A46EB
:1051D00003C23746FFF77CFD7FE6104B206861680D
:1051E00003C37AE64F46B9F1000F04D0B8F1000FBF
:1051F0003FF4F5AEE5E6012262F3071C83F806C032
:1052000093E803000193FFF763FD019B1846FFF746
:1052100037FB019B9B79A3715FE600BFDC93FF1F07
:10522000F0B589B08DE803006846FFF7E1FD074659
:10523000002839D0BDF804309DF800109DF80120F9
:10524000FBB9374E374C33782078984217D0364D1B
:105250002F460EE0237807EBC30393E80300FFF724
:1052600037FD20783378013000F00700834220704A
:1052700005D005EBC000FFF7BBFD0028EAD109B05F
:10528000F0BD8DF808108DF80920BDF808204FF604
:10529000FF739A42D5D0224E224C9DE80300FFF7BF
:1052A00017FD33782078D0E79DE80300BDF804208F
:1052B0009DF800509DF8014006AB83E80300ADF86F
:1052C0001C208DF818508DF81940002AB9D08DF89F
:1052D00010508DF81140BDF810104FF6FF7291423A
:1052E000AFD00F4E0F4C32782078511C01F00701DF
:1052F00081420CD031700C4D93E8030005EBC202E3
:1053000082E80300FFF7ECFC337820789DE7FFF795
:105310009FFC064B377027701F605F60AFE700BFD0
:10532000E593FF1FE493FF1F9C93FF1FDC93FF1F78
:105330002DE9F0418046002850D00026354601274F
:1053400098F80000752808F101042AD02ED8732897
:1053500067D8042861D201284DD0022877D198F867
:10536000010000F12003DBB2072B08F102086BD823
:1053700000F0070007FA00F0C0B200F061FA00F098
:105380006FF9002DDCD02C460120FCF7F9F9631EE3
:1053900013F0FF04F8D198F80000752808F1010413
:1053A000D4D198F8015008F10208EAE7782817D01C
:1053B0000AD876281AD077284DD13046A04600F07A
:1053C00027FA00F04DF9DCE7A0F184036F2B40D8F9
:1053D00000F07F00FFF7ECF9A046D2E7BDE8F081CE
:1053E00000F01EFAA04600F03BF9CAE700F0F8F919
:1053F000A0460646C5E798F8013003F12002D2B274
:10540000072A08F102081BD803F007039840C0B22E
:1054100000F00EFA00F024F9B3E7FFF7F1F8A04628
:10542000AFE798F8013008F10208002BA9D01C461C
:105430000120FCF7A5F9631E13F0FF04F8D1A0E7E3
:105440001846FFF7DDF89CE7FFF7B2F999E7BDE8EA
:10545000F081BDE8F081BDE8F08100BF00000000F0
:10546000704700BF000000000000000000000000C6
:1054700008B5044B186000F0A3FBBDE80840FFF737
:10548000CFBB00BFEC93FF1F000000000000000036
:10549000054A08B5136803431846136000F090FBF3
:1054A000BDE80840FFF7BCBBEC93FF1F0000000005
:1054B000054A08B5136803401846136000F080FBE6
:1054C000BDE80840FFF7ACBBEC93FF1F00000000F5
:1054D000054A08B5136843401846136000F070FB96
:1054E000BDE80840FFF79CBBEC93FF1F00000000E5
:1054F00008B5054A00231846136000F069FBBDE8B3
:105500000840FFF78DBB00BFE893FF1F00000000BD
:1055100008B501238340044A1846136000F058FB85
:10552000BDE80840FFF77CBBE893FF1F00000000C8
:10553000064908B50A6801238340134318460B60E7
:1055400000F046FBBDE80840FFF76ABBE893FF1F89
:10555000074908B50A680123834022EA0303184675
:105560000B6000F035FBBDE80840FFF759BB00BFFA
:10557000E893FF1F00000000000000000000000092
:10558000064908B50A6801238340534018460B605A
:1055900000F01EFBBDE80840FFF742BBE893FF1F89
:1055A000054A08B5136803431846136000F010FB62
:1055B000BDE80840FFF734BBE893FF1F0000000080
:1055C000054A08B5136803401846136000F000FB55
:1055D000BDE80840FFF724BBE893FF1F0000000070
:1055E000054A08B5136843401846136000F0F0FA06
:1055F000BDE80840FFF714BBE893FF1F0000000060
:10560000704700BF00000000000000000000000024
:1056100030B5104A104B15681B6883B01D43ADF8B8
:1056200004001F2402E014F1FF340CD325FA04F324
:10563000DB07F8D5E0B2019900F0F2F980B2012859
:10564000F1D003B030BD0199002000F0E9F903B0BA
:1056500030BD00BFEC93FF1FE893FF1F0000000068
:1056600030B40F4B0F4A1049104D1B781278086860
:1056700029781343037079B10B43037000F10F04D1
:105680000346002213F8011F09B10132D2B2A3422E
:10569000F8D10AB100232B7030BCFEF779BE00BFF1
:1056A000F093FF1FF293FF1F3486FF1FF193FF1F3C
:1056B000F0B41D4B1B7813B11C4B1B78EBB91C4B82
:1056C0001968FF2500234C1C01E00E2B0ED014F8A6
:1056D000012F9042DFB26EB203F101030BD001360D
:1056E000F3D1002A08BF3D460E2BF0D16DB26B1CE2
:1056F00001D00D44A870F0BC7047C3080E2B08D928
:105700000C4B1B78DA07F6D50146F0BC0A4800F0CE
:1057100067BC074A1268134400F007005978012259
:1057200082400A435A70E6E70086FF1F3186FF1F5A
:105730003486FF1F0494FF1FE88200000000000071
:1057400010B4174B1B7813B1164B1B7873B9164B5B
:105750001C680021631C0F3413F8012F824208BF1C
:105760001970A342F8D15DF8044B7047C3080E2BA3
:1057700009D90E4B1B78DB07F5D501465DF8044BC4
:105780000B4800F02DBC084A1268134400F00700D3
:1057900059780122824021EA02025A70E3E700BFF1
:1057A0000086FF1F3186FF1F3486FF1F0494FF1FF2
:1057B000088300000000000000000000000000005E
:1057C000044B1B68002103F10F0203F8011F9342F1
:1057D000FBD170473486FF1F00000000000000006E
:1057E000014B1878704700BFF293FF1F00000000C4
:1057F000024A137818431070704700BFF293FF1FDE
:10580000024A137823EA000010707047F293FF1FDA
:10581000014B1870704700BFF293FF1F000000009B
:10582000014B00221A707047F293FF1F0000000026
:10583000024A137818431070704700BFF093FF1F9F
:10584000024A137823EA000010707047F093FF1F9C
:10585000014B00221A707047F093FF1F00000000F8
:10586000014B1870704700BFF193FF1F000000004C
:10587000014B00221A707047F193FF1F00000000D7
:10588000BC2808B508D8A82819D2A4284AD80428C2
:1058900001D2012810D108BDE7283ED8E028FAD26D
:1058A000BF2809D1FFF7D4F93220FBF769FF00F0D8
:1058B0002FFC4FF0000008BD4FF0000008BD42D0A3
:1058C000A9283DD0AA2844D0AB2836D0AC2843D054
:1058D000AD2844D0AE2845D0AF2846D0B12847D017
:1058E000B02848D0B22849D0B3284AD0B4284BD0E9
:1058F000B5284CD0B6284DD0B7284ED0B82852D0B5
:10590000B9284DD0BA2854D0BB284FD0BC2844F277
:105910002A6018BF4FF4884008BDF028CCD340F46B
:10592000A04008BDA52811D044F2820244F28303AE
:10593000A6280CBF1046184608BD44F2B54008BD65
:1059400044F2E94008BD44F2E24008BD44F281005F
:1059500008BD44F2EA4008BD44F2B64008BD44F236
:10596000B34008BD44F2B44008BD44F2B74008BD9E
:1059700044F2CC4008BD44F2CD4008BD44F283500F
:1059800008BD44F28A5008BD44F2925008BD44F26A
:10599000945008BD44F2216008BD44F2236008BD64
:1059A00044F2256008BD44F2246008BD44F227603B
:1059B00008BD44F2266008BD0000000000000000A1
:1059C0000020704700000000000000000000000000
:1059D000704700BF00000000000000000000000051
:1059E000C1F30723064A00EBC00003EBC30300EB3F
:1059F000C000184452FA81F182B0085C02B07047CE
:105A0000E88100000000000000000000000000002D
:105A1000024BC03833F81000704700BFE48100002B
:105A200000B583B0ADF804100199FFF7D9FFDF2866
:105A3000034611D8C02843D2312863D01FD8292863
:105A400037D02A2848D13A4A1278520613D54FF057
:105A5000310003B05DF804FBE32843D01CD9E628ED
:105A600057D0E72838D1324A1278C2F3C000002854
:105A70005BD1D106EDD4184603B05DF804FB39289C
:105A800021D082281FD0352826D1294A12789206A3
:105A9000F1D54FF02900DCE7E0282CD0E2281BD11B
:105AA000234A12785107E6D5D0063BD54FF00000C7
:105AB000CFE71F4A12789006DDD54FF03500C8E7D2
:105AC000FFF7A6FFC5E71A4A1278D10701D492075B
:105AD00002D54FF0E000BCE71846FFF7D1FE03B057
:105AE0005DF804FB124A1278C2F380000028C0D08F
:105AF0004FF0E200ADE70E4A1278D007BBD54FF069
:105B00003900A6E70A4A12785106B4D54FF02A00A8
:105B10009FE7074A12781107ADD5D006C6D44FF0DB
:105B2000E70096E74FF0E30093E74FF0E60090E7D9
:105B30001094FF1F000000000000000000000000A3
:105B4000030A10B4C4B221091A0941EA041142EA55
:105B50000313C9B2DBB201F0330403F03302A40033
:105B6000920001F0CC0103F0CC0344EA910142EA37
:105B7000930301F0550003F05502400001F0AA0123
:105B8000520003F0AA0340EA510142EA530040EAFE
:105B900001205DF8044B7047000000000000000089
:105BA000704700BF0000000000000000000000007F
:105BB00082B002AB03E9030002B0704700000000AE
:105BC000704700BF0000000000000000000000005F
:105BD000704700BF0000000000000000000000004F
:105BE000FEF7D6BC0000000000000000000000002E
:105BF000704700BF0000000000000000000000002F
:105C00001120FBF7BDBD00BF000000000000000038
:105C1000704700BF0000000000000000000000000E
:105C2000704700BF000000000000000000000000FE
:105C300010B5FFF7EDFFFEF723FAFFF7F1FF0024A1
:105C4000E0B2FEF74DFB013410B9092CF8D110BDBC
:105C5000012010BD00000000000000000000000056
:105C600008B5FFF7DDFDFFF7F3FDFFF7A9FD00F035
:105C7000CFFF0020FEF7CCFB0020BDE80840FEF778
:105C8000D7BB00BF000000000000000000000000C3
:105C90008842F0B54FF0010432D301FB04F4B0FBAD
:105CA000F4F58D42F9D26CB300260CE0002A14BF43
:105CB0004FF0370E4FF0570E75441D7001369CB1F2
:105CC000B0FBF4F53B4604FB15005F1CB4FBF1F49C
:105CD0000EB9002D0BDD092DE8DC4FF0300E7544B8
:105CE0001D700136002CEBD100233B70F0BD0CB1D0
:105CF0001F46E5E75F1C30351D7000233B70F0BD8B
:105D00000546D1E71F46EFE7000000000000000055
:105D10008842F0B54FF0010432D301FB04F4B0FB2C
:105D2000F4F58D42F9D26CB300260CE0002A14BFC2
:105D30004FF0370E4FF0570E75441D7001369CB171
:105D4000B0FBF4F53B4604FB15005F1CB4FBF1F41B
:105D50000EB9002D0BDD092DE8DC4FF0300E754437
:105D60001D700136002CEBD100233B70F0BD0CB14F
:105D70001F46E5E75F1C30351D7000233B70F0BD0A
:105D80000546D1E71F46EFE70000000000000000D5
:105D90002DE9F047DDF820A09AF80040002B0746D7
:105DA000884614BF4FF030094FF020090AF1010670
:105DB000F4B1002A13DD334600E082B113F8011B71
:105DC000013A0029F9D1551E4AB1013D38464946EC
:105DD000C0476B1C002BF8DC9AF8004064B12146E8
:105DE0003846C04716F8014B002CF8D1BDE8F087C3
:105DF000002A02F1FF35E8DCBDE8F0870000000072
:105E00002DE9F04786B08146884616461F4603AD09
:105E1000317839B1252908D001364846C047317854
:105E20000029F7D106B0BDE8F0877378302B3ED05B
:105E300002364FF0000AA3F13001CAB2092A4FF02E
:105E4000000426D96C2B37D0632B5DD053D9732B2C
:105E500047D063D9752B6FD107F1040E38680A213A
:105E600000222B467746FFF753FF00952246534604
:105E700048464146FFF78CFFCAE7A3F157010A29BC
:105E8000E0DC16F8013B04EB840401EB4404A3F1CD
:105E90003001CAB2092AA3F16100F2D90528A3F1A1
:105EA0004102EAD9052ACDD8A3F13701E7E7B37853
:105EB0004FF0010A0336BEE73278632A06F1010685
:105EC00022D048D9732A0CD05ED9752A4DD107F15A
:105ED000040E38680A2100222B467746FFF7D8FEC9
:105EE000C3E73B68009322464846414600230437F7
:105EF000FFF74EFF8CE7252B0CD0582B1FD0002B23
:105F000086D106B0BDE8F0873B1D397848461F466C
:105F1000C0477DE748462521C04779E7642B7FF4D9
:105F200077AF3868002807F104073BDB2B460A21CE
:105F30000022FFF7EDFE98E7782B7FF469AFA3F11D
:105F400058023868B2FA82F2102152092B46FFF744
:105F5000DFFE043789E7252ADCD0582A08D0002A3A
:105F60007FF456AF06B0BDE8F087782A7FF450AFD3
:105F70003868A2F158021021B2FA82F22B46520977
:105F80000437FFF785FE70E7642A7FF441AF386875
:105F9000002807F104070CDB2B460A210022FFF73B
:105FA00077FE62E72D238DF80C3040420DF10D0392
:105FB000BDE72D238DF80C3040420DF10D03ECE7C9
:105FC000024A034B11601860704700BF0894FF1F1E
:105FD0000C94FF1F00000000000000000000000003
:105FE0000FB400B583B004AB0648074953F8042B3F
:105FF000006809680193FFF703FF03B05DF804EB45
:1060000004B070470C94FF1F0894FF1F00000000AD
:10601000704700BF0000000000000000000000000A
:1060200038B5202383F311880F4CFAF769FFA56A6E
:10603000FAF776FF2368A34207D0A2699B689268AB
:106040009A4202D20948FAF70BFF002383F3118822
:106050004FF47A7005FB0000054B0138A3FB0030BC
:10606000C0F38F1038BD00BFD888FF1F2883000001
:10607000D34D62100000000000000000000000008E
:1060800038B5202383F311880E4CFAF739FFA56A3F
:10609000FAF746FF2368A34207D0A2699B6892687B
:1060A0009A4202D20848FAF7DBFE002383F31188F4
:1060B0004FF47A7005FB0000044B0138A3FB00305D
:1060C000800938BDD888FF1F28830000D34D621097
:1060D0000B4B0C499A6A4FF47A7303FB00F000F201
:1060E000E73000B50132A1FB00E0A2EB901003FB0A
:1060F00000F00138A1FB0030C0F38F105DF804FB05
:10610000D888FF1FD34D621000000000000000007F
:1061100008B56420FBF734FB00BE08BD000000009A
:106120002DE9F041054682B00027FEB23046FEF769
:10613000D7F80024804601E0092C22D048FA04F365
:1061400013F0010FE2B204F10104F5D08DF8042040
:106150008DF8056001990020FFF762FC82B2C0F360
:106160000723AA42C0B203F0E00206D013F0C00F2A
:1061700001D0A02AE0D1A842DED1012002B0BDE8C2
:10618000F0810137092FD0D1002002B0BDE8F081A5
:1061900010B504462C20FFF7C3FF00B910BD204600
:1061A000BDE81040FFF7BCBF000000000000000089
:1061B00010B500F01DFA002800F0E5809448FFF7C4
:1061C0000FFF6424FDF75CFF0A20FBF7D9FA631E7A
:1061D00013F0FF04F6D18F48FFF702FF2920FFF7E5
:1061E000D7FF00B110BD2A20FFF7D2FF002840F0F2
:1061F000D5800520FFF7CCFF002840F0D780FFF7BF
:10620000F7FC00F005FA844C20700720FFF7C0FF70
:10621000002840F0CE802078804C00F001FA00F099
:1062200017FA2070E020FFF7B3FF38B12378C3F3EB
:10623000000282F0010262F3000323703920FFF7AD
:10624000A7FF38B12378C3F3400282F0010262F362
:1062500041032370E220FFF79BFF38B12378C3F39B
:10626000800282F0010262F382032370E620FFF7CE
:106270008FFF38B12378C3F3C00282F0010262F3CA
:10628000C3032370E320FFF783FF38B12378C3F300
:10629000001282F0010262F3041323703520FFF72D
:1062A00077FF38B12378C3F3401282F0010262F322
:1062B000451323703120FFF76BFF38B12378C3F308
:1062C000801282F0010262F3861323701120FFF71F
:1062D0005FFF38B12378C3F3C01282F0010262F38A
:1062E000C7132370207800F0BBF923784C4AC3F31E
:1062F000C01327201370FFF74BFF04461E20FFF743
:1063000047FF10B144F00204E4B21F20FFF740FF42
:1063100010B144F00404E4B22020FFF739FF10B1BB
:1063200044F00804E4B22120FFF732FF10B144F03A
:106330001004E4B22220FFF72BFF10B144F0200438
:10634000E4B22320FFF724FF70B144F0400424207E
:10635000E4B2FFF71DFF58B9204600F071F920465E
:10636000BDE81040FFF784B82420FFF711FF68B1A3
:1063700064F07F04E4B2204600F062F92046BDE8F4
:106380001040FFF775B800F01BF917E7002CE3D1B8
:1063900000F04EF9BDE81040FFF76AB800F010F9C0
:1063A0000520FFF7F5FE00283FF429AFFFF7B0FE08
:1063B00025E71B20FFF7ECFE40B12378C3F3400232
:1063C00082F0010262F34103237024E70E20FFF7FD
:1063D000DFFE40B12378C3F3800282F0010262F352
:1063E0008203237017E71020FFF7D2FE237838B11D
:1063F000C3F3C00282F0010262F3C30323700AE711
:10640000C3F3000282F0010262F30003237002E78B
:10641000348300004C8300000494FF1F1094FF1F7E
:106420003186FF1F00000000000000000000000097
:1064300070B5154B154D596818689A68DB6884B0BB
:106440006C460FC46B7899076E460AD40F4944F620
:10645000216301E0013B02D04A78D207FAD504B0AB
:1064600070BD802139220323E971EA72AB7272B6E2
:1064700046F001062846B04762B62B7813F0700349
:10648000E4D02B7004B070BDEC7700000000024037
:106490001F2809D810B5084B5B78DB07044605D5E3
:1064A00004F1A050007810BD00207047FFF7C0FF36
:1064B00004F1A050007810BD000002400000000070
:1064C0001E2809D810B5084B5B78DB07044605D5B4
:1064D00004F1A050008810BD00207047FFF7A8FF0E
:1064E00004F1A050008810BD000002400000000030
:1064F0001F2812D800B50F4B5B78DA0783B00DD593
:1065000000F1A05003788B4204D00A4A01705378FE
:10651000DB07FCD503B05DF804FB70478DE8030092
:10652000FFF786FF9DE8030000F1A05003788B423F
:10653000EBD1EFE700000240000000000000000087
:106540001E2829D800B51B4B5B78DB0783B024D508
:1065500010F0010F00F1A0500AD103888B4204D043
:10656000144A01805378D907FCD503B05DF804FBC9
:1065700003788B4204D00F4A01705378DB07FCD5B7
:106580004378090A8B42F0D00A4A41705378DB07FE
:10659000FCD503B05DF804FB70478DE80300FFF7FE
:1065A00047FF9DE8030010F0010F00F1A050DFD17C
:1065B000D3E700BF00000240000000000000000020
:1065C00008B500204FF6ED61FFF7BAFF0220002169
:1065D000FFF78EFF03200021FFF78AFF0420002130
:1065E000FFF786FF05200021BDE80840FFF780BFC8
:1065F00008B50020FFF764FF4FF6ED63C01AB0FA4C
:1066000080F0400908BD00BF00000000000000004D
:106610000220FFF73DBF00BF0000000000000000A7
:1066200001460220FFF764BF0000000000000000E8
:106630000320FFF72DBF00BF000000000000000096
:1066400001460320FFF754BF0000000000000000D7
:106650000420FFF71DBF00BF000000000000000085
:1066600001460420FFF744BF0000000000000000C6
:106670001B4B1B78D90709D51A4B187800EB800003
:10668000C0F38F007F280BD97F2070479A070AD567
:10669000144B187800EB8000C0F34F007F28F3D82C
:1066A00078B9012070475B0706D40F4B1B7853B1B4
:1066B0000E4A1078834208D30A4B187800EB80000A
:1066C000E0E7C0B2704705207047064A127802EB37
:1066D000820203FB02F393FBF0F080B2D2E700BF2B
:1066E0001194FF1F3986FF1F1994FF1F3A86FF1F61
:1066F000154B1B78D90705D5144B1878800880B145
:10670000C0B270479A0704D5104B1878400840B1C2
:10671000F6E75B0707D50D4B18787F28EFD97F2068
:106720007047012070470A4B1B7853B1094A127811
:106730009342F0D20549087810FB03F393FBF2F083
:10674000EBE70120DCE700BF1194FF1F3C86FF1F31
:106750001994FF1F3886FF1F000000000000000092
:10676000F02808B528D0F1282CD0F2282FD0F32813
:106770001DD0F92831D0FA2834D0FB2838D0FC2895
:106780003CD0F42845D0F52849D0F6284DD0F7283C
:1067900051D0F82855D0FD2835D0FE2857D0FF28F5
:1067A00004D12E4A137843F00403137008BDFFF799
:1067B0005FFF2B4B587008BDFFF75AFF284B404234
:1067C000987008BDFFF754FF254B987008BDFFF780
:1067D0004FFF234B4042587008BDFFF789FF204B05
:1067E000D87008BDFFF784FF1D4B4042D87008BD2C
:1067F000FFF77EFF1A4B4042187108BDFFF778FF84
:10680000174B187108BD154A137843F00103137034
:1068100008BD134A137843F00103137008BD104AF2
:10682000137843F00203137008BD0D4A137843F048
:106830000403137008BD0A4A137843F00803137069
:1068400008BD074A137843F01003137008BD034ACC
:10685000137843F00203137008BD00BF1194FF1FAB
:106860001494FF1F00000000000000000000000062
:10687000F0283FD0F1282CD0F22836D0F32840D091
:10688000F92863D0FA286AD0FB2842D0FC2846D0E9
:10689000F4284DD0F52852D0F6286ED0F72873D0C2
:1068A000F82878D0FD2860D0FE287BD0FF2800F0A3
:1068B0008180444B5A785AB993F9022042B993F92E
:1068C0000330404A23B992F904300BB93E4A1370A1
:1068D00070473C4B93F90220002AEBDD93F901202D
:1068E00000219970002AEAD07047364B5A78110679
:1068F000E1D50BE0334B93F90220002AEEDB5A7806
:10690000D9E7304B5A7851B20029D4DD00225A70B1
:10691000D2E72C4B93F90420002ACBDA04E0294B70
:1069200093F90420002AC5DD00221A715A78C2E7C3
:10693000244B19785A7821F001011970BBE7214BDB
:1069400019785A7821F002011970B4E71D4B93F9B8
:106950000320002AAEDD0022DA705A78ABE7194B2B
:1069600093F90320002AA5DAF5E71848154B0178BA
:106970005A7821F0010101709DE7124B19785A787D
:1069800021F00401197096E70E4B19785A7821F01E
:10699000080119708FE70B4B19785A7821F0100114
:1069A000197088E70948074B01785A7821F00201ED
:1069B000017080E70548034B01785A7821F0040103
:1069C000017078E71494FF1F1994FF1F1194FF1FA3
:1069D00010B5234B1B781B073AD5224C2248FFF7F2
:1069E000FFFA21782148FFF7FBFA2148FFF7F8FA70
:1069F00094F901101F48FFF7F3FA1F48FFF7F0FA68
:106A000094F902101B48FFF7EBFA1B48FFF7E8FA6E
:106A100094F903101748FFF7E3FA1748FFF7E0FA75
:106A200094F904101348FFF7DBFA1448FFF7D8FA7B
:106A3000134B14481978FFF7D3FA1348FFF7D0FA2D
:106A4000124B10481978FFF7CBFA1148FFF7C8FA34
:106A50000448FDF7D5FCFFF7E3FA0E4B188010BD94
:106A60000494FF1F1494FF1F5483000098820000B9
:106A7000788300007C830000948200008083000003
:106A80001994FF1F84830000888300001194FF1F66
:106A9000908400001A94FF1F000000000000000016
:106AA0002DE9F843524B1888FFF712FB51490A7839
:106AB000002A6AD0504B1B7883426DDC4F4C94F80F
:106AC0000180A578E6782779B8F1000F58D11DB973
:106AD00016B9002F00F08580FF2A0FD001320A700E
:106AE0004FFA88F3002B07DDFFF7C2FD5FFA80F84D
:106AF00084F801804FFA88F3002B5FDB6DB2002D24
:106B000004DDFFF7B5FDC5B2A5706DB2002D60DBE9
:106B1000B8F1000F1CD0A578DFF8E090C5B14FFAAE
:106B200088F0F9F757FE30A3D3E90023F9F7B8FE50
:106B3000FAF7CEF889F8010068B2F9F74BFE2AA3FC
:106B4000D3E90023F9F7ACFEFAF7C2F889F802009E
:106B500076B2002E04DDFFF7CBFDC6B2E67076B24A
:106B6000002E23DB7FB2002F04DDFFF7C1FDC7B28B
:106B700027717FB2002F11DBBDE8F843FFF728BF74
:106B8000FF2AADD001320A70AAE71D4B1B7803EB38
:106B900083035B00834291DDBDE8F883FFF7A8FD26
:106BA00040422071BDE8F843FFF712BFFFF7A0FD98
:106BB0007FB24042002FE070D7DCDBE7FFF758FDE3
:106BC0006DB240425FFA80F8002D84F8018098DCB5
:106BD0009CE7FFF74DFD4042A070B8F1000FB7D021
:106BE00099E7BDE8F88300BF666666666666E63FBD
:106BF0001A94FF1F1994FF1F3D86FF1F1494FF1F57
:106C00003B86FF1F000000000000000000000000A5
:106C1000044A0548054900231360137103700B7083
:106C2000704700BF1494FF1F1994FF1F1194FF1F9A
:106C300008B50548FFF7D4F9044805210122BDE84D
:106C40000840FFF7CDB900BF98830000948400008E
:106C50000138052846D8DFE800F00E19242F3A0342
:106C6000214B22481A781144FE29D4BFC9B2FF2112
:106C70001970FFF7B5B91E4B1E481A781144FE294A
:106C8000D4BFC9B2FF211970FFF7AAB91A4B1B482C
:106C90001A781144FE29D4BFC9B2FF211970FFF739
:106CA0009FB9174B17481A781144FE29D4BFC9B2AF
:106CB000FF211970FFF794B9134B14481A78114447
:106CC000FE29D4BFC9B2FF211970FFF789B9104B53
:106CD00010481A781144FE29D4BFC9B2FF21197097
:106CE000FFF77EB9704700BF3886FF1F5085000050
:106CF0003B86FF1FE48400003D86FF1FF4840000F4
:106D00003986FF1F088500003A86FF1F1C8500009A
:106D10003C86FF1F348500000000000000000000DA
:106D20000138052846D8DFE800F00E19242F3A0371
:106D3000214A2248137899423ABF591AC9B2002110
:106D40001170FFF74DB91E4A1E4813788B4286BF5B
:106D5000591AC9B200211170FFF742B91A4A1B48EB
:106D6000137899423ABF591AC9B200211170FFF73E
:106D700037B9174A1748137899423ABF591AC9B216
:106D800000211170FFF72CB9134A14481378994267
:106D90003ABF591AC9B200211170FFF721B9104A40
:106DA0001048137899423ABF591AC9B2002111709C
:106DB000FFF716B9704700BF3886FF1F50850000E7
:106DC0003B86FF1FE48400003D86FF1FF484000023
:106DD0003986FF1F088500003A86FF1F1C850000CA
:106DE0003C86FF1F3485000000000000000000000A
:106DF00010B5014604460548FFF7F2F80120A0400F
:106E0000FEF736FBBDE81040FDF722BF6C850000A1
:106E100038B5831F422B00F2C081DFE813F0510028
:106E200062007200BE01BE012101BE01BE01260149
:106E3000BE013A014E01BE01BE01BE01BE015C01B0
:106E4000BE01BE017C01BE019001BE01A201AD01E7
:106E5000AD01AD01AD01AD01AD01AD01AD01AD01C2
:106E6000B301BE01B301BE01BE01BE01BE01BE0140
:106E7000BE01BE01BE01BE01BE01BE01B301BE0125
:106E8000BE012101BE01B801B801B801B801B801C5
:106E9000B801B801B801B801B301BE01BE01BE011D
:106EA000BE014300FDF7D4FEC148FFF799F84FF447
:106EB0007A70FAF765FC0124FFF72AF9204638BDFD
:106EC000BC4ABD48137803F0F1036FF3000313705D
:106ED000FFF786F8B948FFF783F8B94B01241C7017
:106EE000ECE7B44D2C7814F0010400F0D081B548E3
:106EF000FFF776F82B7803F0F1036FF300032B70A4
:106F0000DCE7B148FFF76CF8B048FFF769F8FFF726
:106F10008FFB0146AE48FFF763F8AE48FFF760F815
:106F2000FFF776FB0446AC48FFF75AF82146AB481A
:106F3000FFF756F8A748FFF753F8A948FFF750F8AE
:106F400004F00101A248FFF74BF8A248FFF748F808
:106F5000A448FFF745F8C4F340019D48FFF740F807
:106F60009C48FFF73DF8A048FFF73AF8C4F38001CA
:106F70009748FFF735F89748FFF732F89B48FFF737
:106F80002FF8C4F3C0019248FFF72AF89148FFF7A1
:106F900027F8FFF75DFB04469548FFF721F82146E7
:106FA0008E48FFF71DF88B48FFF71AF89148FFF756
:106FB00017F804F001018648FFF712F88548FFF73B
:106FC0000FF88D48FFF70CF8C4F340018048FFF735
:106FD00007F88048FFF704F88848FFF701F8C4F382
:106FE00080017B48FEF7FCFF7A48FEF7F9FF8448F2
:106FF000FEF7F6FFC4F3C0017548FEF7F1FF7548D0
:10700000FEF7EEFF7F48FEF7EBFFC4F30011704878
:10701000FEF7E6FF6F48FEF7E3FF7B48FEF7E0FF71
:10702000C4F340116A48FEF7DBFF6A48FEF7D8FF59
:107030007648FEF7D5FFC4F380116548FEF7D0FF10
:107040006448FEF7CDFF7248FEF7CAFFC4F3C011D3
:107050005F48FEF7C5FF5F48FEF7C2FF01242DE73A
:107060006C48FEF7BDFF012428E7524D2B7883F0D2
:107070000404C4F3800464F382032B70002C00F03A
:1070800001816548FEF7ACFF2B7843F001032B70BC
:1070900014E7484D2B7883F00804C4F3C00464F36C
:1070A000C3032B70002C00F0E8805C48FEF798FFCB
:1070B0002B7843F001032B7000E7FDF7C9FD584B17
:1070C0001C7884F001041C70002C00F0D18055481D
:1070D000FEF786FFF2E65448FEF782FFFDF750F90F
:1070E00001465248FEF77CFF514B52481978FEF793
:1070F00077FF514B51481978FEF772FF484B5048C3
:107100001978FEF76DFFFEF7BBFF01464D48FEF70D
:1071100067FF0124D2E64C48FEF762FF4B48FEF7BA
:107120005FFF4B48FEF75CFF4A48FEF759FF4A48AD
:10713000FEF756FF4948FEF753FF0124BEE61D4DFA
:107140002B7883F00204C4F3400464F341032B70F2
:1071500044B34348FEF744FF2B7843F001032B7000
:10716000ACE64048FEF73CFF00F0DAFAFDF708F91C
:10717000FDF7E6F80124A1E61D38C0B2FFF738FE9E
:1071800001249BE60020FFF733FE012496E6393800
:10719000C0B2FFF72DFE012490E63348FEF720FF32
:1071A00000248BE63148FEF71BFF012486E600BF72
:1071B0007C8700000494FF1F508700007887000040
:1071C0001C94FF1F908700008485000090850000BC
:1071D00084830000C4890000A0850000988200001C
:1071E000B4850000C0850000CC850000D885000073
:1071F000E4850000F8850000148600002C8600005D
:1072000040860000548600006086000074860000FE
:107210009086000098860000CC870000EC87000074
:107220003186FF1F9889000014890000248900001E
:107230000086FF1F40890000F092FF1F5889000060
:107240006C89000080890000088800001888000010
:107250004488000084880000B48800000889000089
:10726000AC87000074850000B0890000BC87000076
:107270000B48FEF7B5FE012420E60A48FEF7B0FEF3
:1072800001241BE60848FEF7ABFE012416E607487A
:10729000FEF7A6FE2B7843F001032B7001240DE6C8
:1072A000A4890000F8870000DC870000A0870000A8
:1072B00000207047000000000000000000000000F7
:1072C00000207047000000000000000000000000E7
:1072D0002DE9F047854D2B78012B064662D058D317
:1072E000022B04D000242C702046BDE8F087C31F79
:1072F0004B2B00F26E81DFE813F09E006C016C01F5
:107300006C01C7006C016C016C016C016C016C01BB
:107310006C011101E8006C016C016C016C016C01E5
:107320006C016C016C016C01F000F000F000F000E9
:10733000F000F0006C016C016C016C016C01E80064
:107340006C016C016C016C016C016C016C016C01D5
:107350006C016C016C016C016C016C01C7006C016B
:107360006C016C016C016C016C016C016C016C01B5
:107370006C016C016C016C016C016C016C016C01A5
:107380006C01CC006C016C01D3006C016C01DA0063
:10739000E100574B1B681B78222B41D0002420466C
:1073A000BDE8F087524B1B681B78222B38D0FFF7C3
:1073B00087FF0446002897D10B3E2D2E00F20E8148
:1073C000DFE816F000010C010C010C010C01F700C4
:1073D0000C010C010C01F4000C010C010C010C015E
:1073E0000C010C010C010C010C010C010C010C0135
:1073F0000C010C010C010C010C010C010C010C0125
:10740000F4000C010C010C010C010C010C010C012D
:107410000C010C010C010C010C010C010C01000110
:10742000FFF746FF044600287FF45EAF3046BDE814
:10743000F047FFF7EDBC2F492F4BDFF8DCC0DFF83A
:10744000D4902E4F2E4D2F484FF00A0E28224FF089
:107450001E0A4FF03208142608240C701A7089F89E
:1074600000A08CF8008087F800E02E70FEF7B8FDD1
:10747000254B1978002940F0B58024480124FEF7F7
:10748000AFFD2046BDE8F087FFF7D2FB1E4B197811
:10749000F0E71D4C0A212078FFF7DAFB2178E9E7B5
:1074A000194C0A212078FFF73BFC2178E2E7164CC3
:1074B00001212078FFF734FC2178DBE7124C012111
:1074C0002078FFF7C5FB2178D4E70F4B1A78002A04
:1074D00000F08D8000221A70CFE7A0F11E06F6B2F0
:1074E0000B4A094B915D1970C4E700BF1C94FF1F44
:1074F0003486FF1F3C86FF1F3886FF1F3986FF1F1B
:107500003A86FF1F448A00001D94FF1F5C8A00001A
:107510008C8300003B86FF1F3D86FF1F3748FEF728
:107520005FFD3748FEF75CFD364B37481978FEF7AC
:1075300057FD3648FEF754FD3548FEF751FD354BF3
:1075400031481978FEF74CFD3048FEF749FD3248C6
:10755000FEF746FD314B2C481978FEF741FD2B48CC
:10756000FEF73EFD2E48FEF73BFD2E4B26481978D0
:10757000FEF736FD2548FEF733FD2B48FEF730FDBC
:107580002A4B21481978FEF72BFD2048FEF728FDED
:107590002748FEF725FD274B1B481978FEF720FDED
:1075A0001A48FEF71DFD244B197863E700232B7062
:1075B0009AE6FFF73DFB2148FEF712FD02232B70F0
:1075C000012491E61E48FEF70BFD1E48FEF708FD5C
:1075D000F6E71D48FEF704FD012485E61A48FEF78C
:1075E000FFFC81E61948FEF7FBFC01247CE6154808
:1075F0000124FEF7F5FC2C7076E600BFB889000088
:10760000C88900003B86FF1F84830000C4890000F6
:10761000DC8900003D86FF1FF08900003986FF1FCE
:10762000008A00003A86FF1F148A00003C86FF1F74
:107630002C8A00003886FF1F1D94FF1FB4890000AC
:107640005087000078870000B0890000548A00004D
:1076500010B5114CF9F7ACFC23880133238013F0EB
:10766000FF0310D062780D4992088A5C9A420FD0CD
:107670000B4A136843F080031360F9F7B1FCBDE8CF
:107680001040FAF7BDBB0220FCF75AFE2378E9E769
:107690000020FCF755FEEBE72094FF1F608A0000F6
:1076A0000000044000000000000000000000000096
:1076B00038B541F238000E4D0E4C2A580E4B42F0B0
:1076C00001022A5000212160A1605A7842F0010293
:1076D0005A701A78302142F002021A705520616007
:1076E0000221FBF755F9236843F04003236038BDBE
:1076F000007004400000044000400640000000000C
:10770000024A136843F0010313607047000004400D
:10771000024A136823F0010313607047000004401D
:10772000024A136883F001031360704700000440AD
:1077300070B4840746D0541E002A41D0CDB203460F
:1077400002E0621EE4B3144603F8015B9A07F8D125
:10775000032C2ED9CDB245EA05250F2C45EA054567
:1077600019D903F110022646103E0F2E42F8105C84
:1077700042F80C5C42F8085C42F8045C02F110022A
:10778000F2D8A4F1100222F00F0204F00F0410321C
:10779000032C13440DD91E462246043A032A46F808
:1077A000045BFAD8221F22F003020432134404F0CF
:1077B00003042CB1C9B21C4403F8011BA342FBD142
:0C77C00070BC704714460346C2E700BFCF
:1077CC0020000000400000008000000000010000CC
:1077DC00000200000004000000050000000600008C
:1077EC006FF07F030370037813F0800FFBD07047AA
:1077FC00E08A00002494FF1F2494FF1F2494FF1F91
:10780C00E08A000000000000000000000000000002
:10781C00E08A0000000000000000000000000000F2
:10782C00E08A0000000000000000000000000000E2
:10783C00E08A0000000000000000000000000000D2
:10784C00E08A0000000000000000000000000000C2
:10785C00E08A0000000000000000000000000000B2
:10786C00E08A0000000000000000000000000000A2
:10787C00947800000088FF1FD888FF1F01000000CB
:10788C00B10D00000000000069646C650000000090
:10789C0053562331000000005356233200000000E1
:1078AC0053562333000000005356233400000000CD
:1078BC0053562335000000005356233600000000B9
:1078CC0053562337000000005356233800000000A5
:1078DC00535623390000000053562331300000006A
:1078EC00535623313100000063685654446F53657E
:1078FC007449000063685654446F5265736574494B
:10790C000000000063685363685265616479490044
:10791C006368536368526561647941686561644961
:10792C0000000000737461636B206F766572666C87
:10793C006F770000636853636857616B65757053AC
:10794C00000000006368546864526573756D654986
:10795C000000000063685468644578697453000043
:10796C00636854686452656C65617365000000005F
:10797C0063685468644372656174655375737065AC
:10798C006E646564490000006368546864536C65F8
:10799C00657053006368546864446F446571756521
:1079AC0075654E6578744900636854686443726504
:1079BC0061746500636854686453757370656E64B4
:1079CC00530000006368537973556E6C6F636B00E2
:1079DC006D61696E00160020040444080C10141824
:1079EC001C202122230000006368537973556E6CB0
:1079FC006F636B0063685265674E65787454687288
:107A0C006561640063684D74784F626A656374499C
:107A1C006E69740063684D74784C6F636B5300002F
:107A2C0063684D7478556E6C6F636B006368537943
:107A3C0073556E6C6F636B006368436F7265416C5A
:107A4C006C6F63416C69676E656449006368537958
:107A5C0073556E6C6F636B0063684865617046723A
:107A6C00656500006368506F6F6C46726565490010
:107A7C006368537973556E6C6F636B006F627147FB
:107A8C006574456D70747942756666657254696D7E
:107A9C00656F7574530000006F6271506F7374469C
:107AAC00756C6C4275666665725300006F62714F3F
:107ABC00626A656374496E69740000006368537987
:107ACC0073556E6C6F636B006F627152656C6561A0
:107ADC007365456D70747942756666657249000010
:107AEC007573625374617274526563656976654926
:107AFC000000000000000000010000005F757362D0
:107B0C005F657030696E00007573625374617274D6
:107B1C005472616E736D6974490000007573625321
:107B2C007461727400000000000000005F757362E5
:107B3C005F6570306F7574006368537973556E6C44
:107B4C006F636B00757362496E6974456E64706F18
:107B5C00696E744900000000757362446973616258
:107B6C006C65456E64706F696E747349000000003B
:107B7C006E76696353657453797374656D48616E81
:107B8C00646C65725072696F7269747900000000E0
:107B9C005F70616C5F6C6C645F7365747061646D55
:107BAC006F64650000000000A12400002128000083
:107BBC00F1280000400040008089FF1F0C92FF1F3D
:107BCC00010000000492FF1F00F00F40160000009F
:107BDC00010000000100000016000000060000007B
:107BEC000600000001000000010000000100000080
:107BFC000100000001000000010000000600000070
:107C0C00060000000100000001000000010000005F
:107C1C00010000000500000005000000010000004C
:107C2C000100000001000000010000000100000044
:107C3C000100000001000000010000000100000034
:107C4C0001000000010000000100000040F00F40A6
:107C5C000600000006000000060000000600000000
:107C6C000100000001000000010000000100000004
:107C7C0001000000010000000100000001000000F4
:107C8C0001000000010000000100000001000000E4
:107C9C0012000000120000000600000006000000A8
:107CAC0001000000010000000100000001000000C4
:107CBC0001000000010000000100000001000000B4
:107CCC0001000000010000000100000001000000A4
:107CDC0080F00F40060000000600000006000000C7
:107CEC000600000006000000060000000600000070
:107CFC000600000006000000060000000600000060
:107D0C00060000000100000001000000010000005E
:107D1C000100000001000000010000000100000053
:107D2C000100000001000000010000000100000043
:107D3C000100000001000000010000000100000033
:107D4C000100000001000000010000000100000023
:107D5C0001000000C0F00F4006000000060000000B
:107D6C0006000000060000000600000006000000EF
:107D7C0006000000060000000100000001000000E9
:107D8C0001000000010000000100000001000000E3
:107D9C0001000000010000000100000001000000D3
:107DAC0001000000010000000100000001000000C3
:107DBC0001000000010000000100000001000000B3
:107DCC0001000000010000000100000001000000A3
:107DDC00010000000100000000F10F40060000004F
:107DEC00060000000100000001000000010000007E
:107DFC000100000001000000010000000100000073
:107E0C000100000001000000010000000100000062
:107E1C000100000001000000010000000100000052
:107E2C000100000001000000010000000100000042
:107E3C000100000001000000010000000100000032
:107E4C000100000001000000010000000100000022
:107E5C00010000000100000001000000090000000A
:107E6C003180000022034300680069006200690051
:107E7C004F005300200054004D004B0020007400B4
:107E8C0065007300740000000900000031800000E0
:107E9C0005010906A10175019508050719E029E7F7
:107EAC0015002501810295057501050819012905A3
:107EBC0091029501750391039578750115002501C3
:107ECC000507190029778102C0000000400000005E
:107EDC006480000012000000807F0000313A000036
:107EEC001135000001380000D135000015000000EC
:107EFC00947F000086000000D47F00000300000087
:107F0C000000000011360000000000000800000016
:107F1C00C492FF1F000000000200000000000000DF
:107F2C0005010902A1010901A10005091901290591
:107F3C0015002501750195058102750395018103D5
:107F4C000501093009311581257F750895028106D7
:107F5C0009381581257F3500450075089501810686
:107F6C00050C0A38021581257F750895018106C01C
:107F7C00C00000001201000200000040EDFE0C0ADF
:107F8C000A000102030100000631FF0974A15375B8
:107F9C0008150026FF00951009758102C00000002D
:107FAC000403090403000000000000000136000077
:107FBC0000000000080000009C92FF1F0000000061
:107FCC00020000000000000009028600050100A06C
:107FDC003209040000010301010009211101000113
:107FEC002240000705810308000A0904010001036F
:107FFC000000000921110100012251000705820334
:10800C00080001090402000103000000092111010C
:10801C000001221500070583031000010904030069
:10802C0001030000000921110100012231000705A4
:10803C00840308000A09040400010300000009215C
:10804C001101000122390007058503100001000011
:10805C0009000000FF7F000005010906A101750160
:10806C009508050719E029E71500250181029501FE
:10807C0075088103950575010508190129059102FB
:10808C0095017503910395067508150026FF0005EB
:10809C0007190029FF8100C0030000000000000048
:1080AC006136000000000000100000004093FF1F2C
:1080BC0000000000020000000000000003000000AF
:1080CC0000000000E1350000000000000800000086
:1080DC008492FF1F0000000002000000000000005E
:1080EC0004000000AC7F00000C000000A481000024
:1080FC0022000000707E0000160000000486FF1FA6
:10810C00510000002C7F000005010980A1018502AF
:10811C00150126B700190129B7751095018100C00A
:10812C00050C0901A10185031501269C0219012AE0
:10813C009C02751095018100C000000063685379A2
:10814C0073556E6C6F636B000900000018800000A3
:10815C000300000000000000F135000000000000EA
:10816C0010000000B092FF1F000000000200000091
:10817C0000000000636F6E736F6C655F666C7573E7
:10818C00685F636200000000310000001481000091
:10819C0009000000E67F00000C0354004D004B006A
:1081AC002000C600390000009C7E00005553422080
:1081BC00636F6E666967757265642E0A0000000055
:1081CC004B6579626F6172642073746172742E0AEC
:1081DC00000000005B735D00F1A10000291E1F2050
:1081EC00212223242526272D2E2A2A2B141A081562
:1081FC00171C180C12132F30314C39041607090AAE
:10820C000B0D0E0F333428284BE11D1B06190511DD
:10821C0010363738E5E5524EE0E3E2652C2C2C2C79
:10822C00C0E6E7E450514F000000000000353A3B37
:10823C003C3D3E3F4041424344452A2A0101010155
:10824C000101010101010101010101010101010112
:10825C000101010101010101010101010101010102
:10826C0001010101010101010101010101010101F2
:10827C0001010101010101010000000000000000EA
:10828C00626F756E6365213A20000000253032580C
:10829C00000000000A722F6320303132333435363F
:1082AC003738394142434445460A000025303136BF
:1082BC00620000006B6579626F6172645F72657059
:1082CC006F72743A200000002530325820000000F4
:1082DC004C45443A20253032580A00006164645FF2
:1082EC006B65795F6269743A2063616E27742061F3
:1082FC0064643A20253032580A00000064656C5FD3
:10830C006B65795F6269743A2063616E27742064CF
:10831C00656C3A20253032580A00000063685379A6
:10832C0073556E6C6F636B00626F6F746D61676910
:10833C0063207363616E3A202E2E2E200000000005
:10834C00646F6E652E0A00006D6F7573656B6579D1
:10835C00205B62746E7C782079207620685D2872B0
:10836C0065702F61636C293A205B00007C00000073
:10837C00256400005D280000257500002F0000001A
:10838C000102030405060708090000000A092D2054
:10839C004D6F7573656B6579202D0A4553432F71AD
:1083AC003A09717569740A313A0964656C61792806
:1083BC002A31306D73290A323A09696E7465727606
:1083CC00616C286D73290A333A096D61785F73709B
:1083DC006565640A343A0974696D655F746F5F6D25
:1083EC0061780A353A09776865656C5F6D61785F0D
:1083FC0073706565640A363A09776865656C5F74F5
:10840C00696D655F746F5F6D61780A0A703A097007
:10841C0072696E742076616C7565730A643A0973BF
:10842C0065742064656661756C74730A75703A09BD
:10843C002B310A646F776E3A092D310A70677570AB
:10844C003A092B31300A7067646F776E3A092D3117
:10845C00300A0A7370656564203D2064656C746134
:10846C00202A206D61785F7370656564202A20284E
:10847C00726570656174202F2074696D655F746F0F
:10848C005F6D6178290A0000776865726520646504
:10849C006C74613A20637572736F723D25642C2085
:1084AC00776865656C3D25640A536565206874744E
:1084BC00703A2F2F656E2E77696B697065646961F0
:1084CC002E6F72672F77696B692F4D6F7573655FB0
:1084DC006B6579730A0000006D6B5F64656C617984
:1084EC00203D2025640A00006D6B5F696E74657217
:1084FC0076616C203D2025640A0000006D6B5F6D79
:10850C0061785F7370656564203D2025640A000006
:10851C006D6B5F74696D655F746F5F6D6178203D25
:10852C002025640A000000006D6B5F776865656C40
:10853C005F6D61785F7370656564203D2025640A0A
:10854C00000000006D6B5F776865656C5F74696D2A
:10855C00655F746F5F6D6178203D2025640A0000B3
:10856C004C25640A00000000536C656570204C4576
:10857C004420746573740A006565636F6E66696781
:10858C003A0A000064656661756C745F6C617965AC
:10859C00723A200064656275675F636F6E66696727
:1085AC002E7261773A2000002E656E61626C653A1E
:1085BC00200000002E6D61747269783A2000000072
:1085CC002E6B6579626F6172643A20002E6D6F7547
:1085DC0073653A20000000006B65796D61705F6314
:1085EC006F6E6669672E7261773A20002E73776121
:1085FC00705F636F6E74726F6C5F636170736C6FBE
:10860C00636B3A20000000002E636170736C6F6323
:10861C006B5F746F5F636F6E74726F6C3A200000E7
:10862C002E737761705F6C616C745F6C6775693AFF
:10863C00200000002E737761705F72616C745F7242
:10864C006775693A200000002E6E6F5F6775693A96
:10865C00200000002E737761705F67726176655F32
:10866C006573633A200000002E737761705F62615E
:10867C00636B736C6173685F6261636B737061636E
:10868C00653A20002E6E6B726F3A20000A092D207D
:10869C004D61676963202D0A643A096465627567E8
:1086AC000A783A096465627567206D61747269783D
:1086BC000A6B3A096465627567206B6579626F6154
:1086CC0072640A6D3A096465627567206D6F757323
:1086DC00650A763A0976657273696F6E0A733A09A0
:1086EC007374617475730A633A09636F6E736F6C9C
:1086FC0065206D6F64650A302D343A096C617965BB
:10870C0072302D34284631302D4634290A5061758B
:10871C00733A09626F6F746C6F616465720A653AC3
:10872C0009656570726F6D0A6E3A094E4B524F0AAD
:10873C007A3A09736C656570204C454420746573F6
:10874C00740A00000A092D20436F6E736F6C65204C
:10875C002D0A4553432F713A09717569740A6D3AA4
:10876C00096D6F7573656B65790A0000433E2000D7
:10877C000A0A626F6F746C6F616465722E2E2E2004
:10878C00000000000A64656275673A206F66660A2D
:10879C00000000000A64656275673A206F6E0A007B
:1087AC000A6D61747269783A206F6E0A00000000DD
:1087BC000A6D61747269783A206F66660A0000006F
:1087CC000A6B6579626F6172643A206F6E0A000001
:1087DC000A6B6579626F6172643A206F66660A0093
:1087EC000A6D6F7573653A206F6E0A000A6D6F75AE
:1087FC0073653A206F66660A000000000A092D2096
:10880C0056657273696F6E202D0A00004445534300
:10881C003A2022544D4B206B6579626F6172642053
:10882C006669726D77617265206F76657220436838
:10883C006962694F53220A005649443A20307846FF
:10884C004545442822544D4B2229205049443A2076
:10885C00307830413043282243686962694F532095
:10886C00544D4B20746573742229205645523A207E
:10887C003078303030410A004255494C443A206639
:10888C003766616264362D646972747920283039D8
:10889C003A30353A3131204F637420203120323058
:1088AC003136290A000000004F5054494F4E533ABC
:1088BC002043484942494F5320424F4F544D414762
:1088CC004943204D4F5553454B455920455854521B
:1088DC00414B455920434F4E534F4C4520434F4D30
:1088EC004D414E44204E4B524F20424F4F544C4F13
:1088FC00414445525F53495A450A00004743433AA5
:10890C0020342E392E3300000A092D205374617443
:10891C007573202D0A000000686F73745F6B6579A6
:10892C00626F6172645F6C65647328293A20255804
:10893C000A0000006B6579626F6172645F70726F20
:10894C00746F636F6C3A2025580A00006B6579626E
:10895C006F6172645F69646C653A2025580A000087
:10896C006B6579626F6172645F6E6B726F3A202512
:10897C00580A000074696D65725F72656164333208
:10898C0028293A202530346C580A00004E4B524F9F
:10899C003A206F6E0A0000004E4B524F3A206F6621
:1089AC00660A00003F0000004D3E20000A092D2001
:1089BC0056616C756573202D0A000000313A2064F5
:1089CC00656C6179282A31306D73293A20000000DA
:1089DC00323A20696E74657276616C286D73293A2F
:1089EC0020000000333A206D61785F737065656418
:1089FC003A200000343A2074696D655F746F5F6DC6
:108A0C0061783A2000000000353A20776865656C83
:108A1C005F6D61785F73706565643A2000000000DB
:108A2C00363A20776865656C5F74696D655F746F45
:108A3C005F6D61783A20000073657420646566612F
:108A4C00756C740A000000004D25643E2000000087
:108A5C004D3E00000000000000000000000000017E
:108A6C000204060A0F17202C3A4A5D71879DB3C782
:108A7C00DAE9F5FCFFFCF5E9DAC7B39D87715D4ACD
:108A8C003A2C20170F0A0604020100000000000017
:048A9C0000000000D6
:108AA000010000001603300078004400450041003A
:108AB000440042004500450046000000613B0000C4
:108AC000713B0000713C0000113D0000713D000051
:108AD00005010000F493FF1F280A141E083200004D
:0400000300000411E4
:00000001FF
